:100000000C9432020C944D020C944D020C944D024F
:100010000C944D020C944D020C944D020C944D0224
:100020000C944D020C94B40D0C944D020C94950D4F
:100030000C94AC180C944D020C944D020C944D028F
:100040000C944D020C944D020C945D0C0C944D02DA
:100050000C94FD040C944D020C94C7040C944D02B6
:100060000C94200F0C944D020C94D6170C944D0256
:100070000A0D466C69676874436F6E74726F6C0A20
:100080000D48617264776172653A25642E25640AB1
:100090000D536F6674776172653A5625642E256438
:1000A000256320000A0D3D3D3D3D3D3D3D3D3D3D2F
:1000B0003D3D3D3D3D3D3D3D3D3D3D3D3D3D3D3D70
:1000C0003D3D3D3D000A0D496E69742E2045455069
:1000D000524F4D3A2047656E6572696572652044DE
:1000E000656661756C742D506172616D65746572C1
:1000F0002E2E2E000A0D414343206E696368742042
:1001000061626765676C696368656E21000A0D420C
:10011000656E75747A6520506172616D6574657283
:100120007361747A202564000A0D4162676C656909
:100130006368204C756674647275636B73656E7367
:100140006F722E2E004F4B0A0D000A0D5374657509
:100150006572756E673A200048656164696E67482C
:100160006F6C64004E65757472616C000A0A0D0054
:100170002E005B25695D005B25695D002B204D69C4
:100180006B726F4B6F70746572202B0048573A5634
:1001900025642E25642053573A25642E2564256353
:1001A0000053657474696E673A20256420002863E3
:1001B0002920486F6C676572204275737300486F21
:1001C0006568653A202020202025356900536F6C32
:1001D0006C486F6568653A20253569004C75667412
:1001E000647275636B3A20253569004F666620207E
:1001F000202020203A20253569004B65696E652056
:100200000048F668656E726567656C756E670061BB
:100210006B742E204C616765004E69636B3A202039
:100220002020202025356900526F6C6C3A20202058
:10023000202020253569004B6F6D706173733A2063
:100240002020253569004B313A25346920204B3276
:100250003A25346920004B333A25346920204B3449
:100260003A25346920004B353A25346920204B3635
:100270003A25346920004B373A25346920204B3821
:100280003A25346920004E693A2534692020526F9E
:100290003A253469200047733A253469202047699C
:1002A0003A253469200050313A25346920205032F3
:1002B0003A253469200050333A25346920205034DF
:1002C0003A25346920004779726F202D2053656EDE
:1002D000736F72004E69636B2025346920282533C3
:1002E000692900526F6C6C202534692028253369F8
:1002F000290047696572202534692028253369293A
:10030000004E69636B202534692028253369290054
:10031000526F6C6C202534692028253369290047E9
:1003200069657220253469202825336929004143F5
:1003300043202D2053656E736F72004E69636B20EE
:1003400025346920282533692900526F6C6C2025DB
:10035000346920282533692900486F6368202534D3
:1003600069202825336929005370616E6E756E67A8
:100370003A202025356900456D70662E5065676509
:100380006C3A253569004B6F6D70617373202020C6
:1003900020202020005269636874756E673A20201F
:1003A000253569004D657373776572743A20202591
:1003B00035690053746172743A202020202025355D
:1003C0006900506F7469313A202025336900506FFD
:1003D0007469323A202025336900506F7469333ACA
:1003E000202025336900506F7469343A202025336A
:1003F0006900536572766F202000536574706F69D1
:100400006E742020253369005374656C6C756E67BB
:100410003A202533690052616E67653A2533692DAC
:100420002533690045787465726E436F6E74726F20
:100430006C2020004E693A2534692020526F3A25FD
:100440003469200047733A253469202047693A25EA
:100450003469200048693A253469202043663A25EA
:100460003469200011241FBECFEFD0E1DEBFCDBF25
:1004700013E0A0E0B1E0E6EAF8E802C005900D92D2
:10048000AE3AB107D9F718E0AEEAB3E001C01D9269
:10049000A034B107E1F70C94BB020C940000FB01FF
:1004A000863008F085E0489FD0011124AC59BF4F39
:1004B000842F9927019724F00E943F440192FACF9C
:1004C0000895282FFB01863008F025E0429FD001D7
:1004D0001124AC59BF4F842F9927019724F0019024
:1004E0000E944744FACFA2E0B0E0022E0E944744A7
:1004F0000895A2E0B0E09D010E943F44802D863027
:1005000028F082E0D901082E0E94474499270895D7
:1005100080916507E82FFF27EE0FFF1FE75CF84F7C
:10052000808191818D5E9F4F14F010920201808135
:1005300091818A5B9F4FBCF480910201882399F4DA
:1005400081E080930201809136068F5F80933606AA
:10055000853038F088EE93E09093CE038093CD03FE
:1005600002C00E94471B809136069927909304078A
:10057000809303070895CFEFD0E1DEBFCDBF14B85D
:1005800015B897EEE92E93E0F92E8EEC9FEFE80E6A
:10059000F91EF7FEFACF88EEE82E83E0F82E189BBE
:1005A00002C08BE001C08AE08093010181E887B935
:1005B0008FEF88B98BE184B981E085B98EE38AB980
:1005C000579A87EF8BB984B7877F84BF809160008B
:1005D0008861809360001092600080ED97E09093B6
:1005E000CE038093CD031092290410922804109218
:1005F0003E0710923D0710922B0410922A0410928D
:100600002D0410922C04809101018A3011F4289855
:1006100001C0289A0E94440D0E9456080E94971813
:100620000E94D20E0E949F170E94C73F789410929A
:10063000260685E48093270687E0809328068CE6CB
:1006400090E09F938F9385E490E09F938F931F9208
:100650001F92809101016AE00E94CF43892F992760
:100660009F938F93809101010E94CF4399279F937D
:100670008F9380E790E09F938F931F920E94D309FE
:100680008DB79EB70D960FB6F8949EBF0FBE8DBF67
:1006900084EA90E09F938F931F920E94D309299A36
:1006A0000F900F900F9001E010E0D8010E943F449E
:1006B000802D863461F185EC90E09F938F931F929B
:1006C0000E94D3090E949619C0E00F900F900F90DE
:1006D000C23039F0C33019F40E94B71A04C0C430D4
:1006E00010F00E94261A47E465E677E08C2F0E94FE
:1006F0006102CF5FC63060F3A2E0B0E083E0082E75
:100700000E94474486E4D801082E0E944744A4E092
:10071000B0E00E943F44802D853050F084EF90E09F
:100720009F938F931F920E94D3090F900F900F9069
:100730000E94790247E465E677E00E944F020E943A
:10074000790299279F938F938DE091E09F938F93E8
:100750001F920E94D30980916D070F900F900F9008
:100760000F900F9080FF20C088E291E09F938F93BD
:100770001F920E94D30988EE93E00E943B0D7C01FA
:100780000E94D80E0F900F900F90C7010E946B0D22
:100790008823D9F385E491E09F938F931F920E9461
:1007A000D3090F900F900F900E94C21C80910101FD
:1007B0008A3011F4289801C0289A80ED97E0909330
:1007C000CE038093CD0385E5809338068AE491E0DB
:1007D0009F938F931F920E94D30980916D070F9072
:1007E0000F900F9082FF03C088E591E002C084E67D
:1007F00091E09F938F931F920E94D3090F900F90C7
:100800000F908CE691E09F938F931F920E94D309E3
:100810000E94291288E893E190938F0380938E03BE
:1008200081E0809337060F900F900F908091D10355
:10083000882309F4A4C01092D1038091360688233E
:1008400019F00E94880202C00E9430280E940125EF
:10085000209101012A3011F4289801C0289A809132
:100860000303882321F081508093030312C08093F7
:10087000AE038093AF038093420610920C04109253
:100880000B0410920A0410920904109208041092AA
:10089000070480912E04882329F080912E04815032
:1008A00080932E0480918E0390918F03892B01F504
:1008B00085E090E090938F0380938E030E94B91798
:1008C00080910603909107038F5F9F4FF9F4809109
:1008D00025048823D9F080E197E29093CE0380939A
:1008E000CD0380E890E090930703809306030EC049
:1008F00080918E0390918F03019790938F03809343
:100900008E032A3011F4289801C0289A8091D103CF
:10091000882321F080912504882311F40E947C080B
:100920000E94E706C7010E946B0D882341F1809168
:100930007D07282F33278091140390911503821788
:1009400093079CF480910603909107038F5F9F4F5C
:1009500061F480E797E19093CE038093CD0380E02C
:1009600093E090930703809306030E946F4184E015
:100970008093CC0384E190E00E943B0D7C01809148
:10098000CC03882309F052CF0E94B0414FCF1F9271
:100990000F920FB60F9211248F939F93EF93FF93B3
:1009A000809105038823E1F48091C2039091C303F1
:1009B00001969093C3038093C203FC01E850FB4F60
:1009C000E081ED3019F08639910539F41092C303B6
:1009D0001092C20381E080930503E093C60004C037
:1009E0001092C3031092C203FF91EF919F918F91D8
:1009F0000F900FBE0F901F9018951F920F920FB679
:100A00000F9211242F933F934F935F938F939F9354
:100A1000AF93BF93EF93FF9390E08091C6008093D4
:100A2000BD035091C803563910F09093C9038091CB
:100A3000BD038D3009F05FC08091C903823009F099
:100A40005AC09093C903852F99278B5B994FFC015E
:100A5000329740812091C4033091C503241B310992
:100A6000DC0111978C91281B3109C9019F7090936B
:100A7000C5038093C40346E0969587954A95E1F7B0
:100A8000982F935C9093C6032F733070235C209350
:100A9000C7038081981729F48C91281711F491E0ED
:100AA00006C090E08091BA038F5F8093BA03809173
:100AB000BC03882309F06EC0992309F46BC081E060
:100AC0008093BC035093B903E52FFF27EB5BF94FED
:100AD0008DE0808380914706823509F05BC088E114
:100AE00090E02CE00FB6F894A895809360000FBEBC
:100AF000209360004FC02091C903822F9927813035
:100B00009105F9F0823091051CF4892B21F040C049
:100B1000029711F13DC08091BD03833239F4809179
:100B2000BC03882319F481E08093C9038091BD033D
:100B30008093450681E08093C8038091BD03992787
:100B400022C02F5F2093C903E52FFF27EB5BF94FEE
:100B50008091BD03808309C0E52FFF27EB5BF94F30
:100B60008091BD038083563920F45F5F5093C803A2
:100B700002C01092C9032091BD038091C4039091DB
:100B8000C503820F911D9093C5038093C40302C0D7
:100B90001092C903FF91EF91BF91AF919F918F91F7
:100BA0005F914F913F912F910F900FBE0F901F902B
:100BB0001895AC01A0E0B0E09D01A817B90748F472
:100BC000E8EFF4E08191280F311D1196A417B507C5
:100BD000C8F33F70FD01E850FB4FC90156E0969500
:100BE00087955A95E1F7835C80831196FD01E85063
:100BF000FB4F2F733070822F835C8083A750BB4FD5
:100C00008DE08C93109205038091F8048093C600C8
:100C100008951F93CF93DF93382FEA01722F10E0CE
:100C200083E28093F8046093F9043093FA04A3E01C
:100C3000B0E0772309F458C0772311F4972F07C049
:100C4000FE01E10FF11D1F5F9081715011F4472FDC
:100C50000EC0FE01E10FF11D1F5F4081715039F0A0
:100C6000FE01E10FF11D1F5F6081715001C0672F10
:100C7000FD01E850FB4F892F86958695835C808324
:100C80001196FD01E850FB4F892F992783709070D2
:100C900024E0880F991F2A95E1F755279A0194E0DF
:100CA000369527959A95E1F7822B835C8083119680
:100CB000FD01E850FB4F4F705070440F551F440F1B
:100CC000551F862F992726E0969587952A95E1F757
:100CD000842B835C80831196FD01E850FB4F6F737A
:100CE000635C60831196A5CFCD010E94D905DF9189
:100CF000CF911F9108951F93CF93DF93EC0110E0E4
:100D0000662309F460C0A22FBB271297E42FFF27A8
:100D1000EB5BF94F30813D534F5FE42FFF27EB5BD7
:100D2000F94F50815D534F5FE42FFF27EB5BF94F85
:100D300070817D534F5FE42FFF27EB5BF94FE0811C
:100D4000ED534F5F842F9927A817B907E4F1832F3C
:100D50009927880F991F880F991F352F32953F705B
:100D6000382B852F99278F709070F4E0880F991F8A
:100D7000FA95E1F7572F56955695582B872F9927B7
:100D80008370907076E0880F991F7A95E1F78E2B2B
:100D900061506F3FC1F0FE01E10FF11D30831F5F15
:100DA00061506F3F81F0FE01E10FF11D50831F5F25
:100DB00061506F3F41F0FE01E10FF11D80831F5F25
:100DC000662309F0A3CFDF91CF911F910895CF93B0
:100DD000DF93CDB7DEB724970FB6F894DEBF0FBE12
:100DE000CDBF8091BC03882309F445C1809147069B
:100DF00099278836910509F494C089369105C4F481
:100E00008236910509F462C08336910544F48B342F
:100E1000910559F18136910509F44CC02AC18336F8
:100E2000910509F467C08736910509F4B2C021C164
:100E3000813791054CF48C3691050CF0D4C08B367B
:100E4000910509F492C015C18437910509F484C055
:100E5000853791052CF48137910509F49EC009C1AD
:100E60008637910509F491C004C12091B90343E08C
:100E700062E0CE0101960E947B0689819A8190935F
:100E8000410480934004809140049091410420915A
:100E90003E0430913F04821B930B845E9D4F68E6B5
:100EA00071E00E94EF43845B904090933D048093F7
:100EB0003C04DFC02091B90343E062E0CE01039619
:100EC0000E947B068B81809304035BC02091B90351
:100ED00043E06BE088E396E00E947B068091F50397
:100EE00090913A06892B8093F50380914106809377
:100EF0001D07BFC02091B90343E06BE088E396E093
:100F00000E947B068091F50390913A06892B80938D
:100F1000F5038091410680931D0781E08093BF0314
:100F200030C02091B90343E062E0CE0103960E94F5
:100F30007B068091F5039B81892B8093F5038C813F
:100F40008F3F21F481E08093B60302C01092B60374
:100F500081E08093C0038DC02091B90343E064E039
:100F600082EB93E00E947B060CC02091B90343E022
:100F700064E08EEA93E00E947B068091B103809347
:100F80001D078FEF8093030374C081E08093BE033D
:100F900070C081E08093C1036CC02091B90343E02D
:100FA00062E0CE0103960E947B06809105038823B0
:100FB000E1F38B818F3F61F0863010F085E08B8309
:100FC00047E465E677E08B810E944F028B8102C087
:100FD0000E94790227E445E657E06091F704855BBB
:100FE0000E94090646C02091B90343E067E485E604
:100FF00097E00E947B068091470647E465E677E02C
:101000008B560E946102A2E0B0E0809147068B56A9
:10101000082E0E944744809190079927AA27BB2752
:10102000BC01CD0124EC39E040E050E00E94B04327
:10103000DC01CB018093880390938903A0938A03FA
:10104000B0938B03809191079927AA27BB27BC01F6
:10105000CD010E94B043DC01CB01809384039093C7
:101060008503A0938603B09387030E9479020E94B0
:10107000471B1092BC0324960FB6F894DEBF0FBE38
:10108000CDBFDF91CF910895CF93C82F8A3019F447
:101090008DE00E9444088091C00085FFFCCFC09382
:1010A000C60080E090E0CF910895089588E1809394
:1010B000C1008091C00082608093C0008091C10017
:1010C00080688093C1008091C10080648093C100DA
:1010D0008AE28093C40088EC90E00E943B0D9093DC
:1010E0002506809324068CED90E00E943B0D9093A2
:1010F000440680934306089580910503882309F4EC
:10110000F7C08091C103882371F080910503882383
:1011100051F02BE048E356E06091F70487E40E9429
:1011200009061092C10380914306909144060E94E3
:101130006B0D882309F44CC080910503882309F4C2
:1011400047C080917A0490917B04A0917C04B09177
:101150007D04BC01CD012CE630E040E050E00E946F
:10116000244430933106209330068091720490918C
:101170007304A0917404B0917504BC01CD012CE6F8
:1011800030E040E050E00E94244430933306209346
:101190003206809116048093340680911504809362
:1011A000350628E040E356E06091F70487E70E94A7
:1011B000090680913606853018F086E08093360661
:1011C00083E690E00E943B0D909344068093430693
:1011D00080912406909125060E946B0D882321F4AE
:1011E0008091BF038823B1F080910503882391F09B
:1011F00022E44BED56E06091F70484E40E94090676
:101200001092BF038AEF90E00E943B0D9093250659
:1012100080932406609104036F3F91F0862F9927F5
:1012200034E0880F991F3A95E1F78D5F9E4F605D1E
:1012300020E1AC0181E40E9409068FEF8093040352
:1012400090911D079923A1F080910503882381F0D7
:1012500083E28093F8049093F9048DE08093FA047C
:101260001092050310921D078091F8048093C60028
:101270008091C003882351F180910503882331F1C7
:101280000E9432121092C0033091B703832F8F5FF8
:101290008093B703843021F06091B603662359F040
:1012A00026E149E357E060E084E30E9409068FEFFE
:1012B0008093B7030BC024E1829FC00111248A5E92
:1012C0009C4FAC01832F8F5C0E9409068091BE0366
:1012D000882371F080910503882351F02AE046E2CB
:1012E00056E06091F70486E50E9409061092BE035D
:1012F0000895982F80911E07813069F48091F6033C
:10130000E82FFF27EA5EFC4F90838F5F8093F60300
:1013100021E030E005C0892F0E944408282F3327A0
:10132000C90108950F931F93CF93DF938C01EB01B5
:10133000672B39F0F80181918F010E94790921977B
:10134000C9F7DF91CF911F910F9108950F931F93CC
:10135000CF93DF938C01EB01672B41F0F8010F5F16
:101360001F4F84910E9479092197C1F7DF91CF9196
:101370001F910F910895CF93C82F181634F480E26F
:101380000E947909C1501C16D4F3CF910895CF93D0
:10139000C82F181634F480E30E947909C1501C1636
:1013A000D4F3CF9108952F923F924F925F926F9214
:1013B0007F928F929F92AF92BF92CF92DF92EF92E5
:1013C000FF920F931F93CF93DF93CDB7DEB7E097D4
:1013D0000FB6F894DEBF0FBECDBF26968FAD269711
:1013E0002896EEADFFAD28971CA61DA61EA61FA62B
:1013F00080931E07A8E46A2E712C6C0E7D1E5F017F
:10140000C50105C0053239F00894A11CB11CF501D5
:1014100004910023B9F7B501681B790B11F00E9404
:10142000A609002309F430C20894A11CB11C55245C
:1014300058AA252C1FEF59A6F5010894A11CB11C30
:101440000491053721F0802F80628837F1F450FE37
:101450000EC0F30124E030E0620E731E80819181A2
:10146000A281B3818CA79DA7AEA7BFA70EC0F30131
:10147000A2E0B0E06A0E7B1E808191819C0144272E
:1014800055272CA73DA74EA75FA7003221F489A5B9
:10149000882391F61BC0033211F438E081C00A3270
:1014A00011F00D3289F40A3251F4F30142E050E0B8
:1014B000640E751E208022200CF0BECF219450E1D6
:1014C000552A8FED5822B8CF0B3211F409A7B4CFAB
:1014D0000E32C1F5F5010894A11CB11C04910A3229
:1014E00079F4F301A2E0B0E06A0E7B1E60817181A5
:1014F000BFEF6F3F7B0714F46FEF7FEF162F9CCF8A
:1015000060E070E0802F80538A30A0F4CB01F3E0DC
:10151000880F991FFA95E1F7860F971F680F791FBB
:10152000600F711D60537040F5010894A11CB11C3F
:101530000491E8CFEFEF6F3F7E0714F46FEF7FEF7A
:10154000162F7FCF003329F454FC76CFF0E25F2AC8
:1015500073CF802F81538930D8F460E070E0CB01E5
:10156000E3E0880F991FEA95E1F7860F971F680F50
:10157000791F600F711D60537040F5010894A11C24
:10158000B11C0491802F80538A3048F3262E59CF06
:10159000083619F424E0522A4FCF0C3619F431E002
:1015A000532A4ACF033661F44E010894811C911CE2
:1015B000F30142E050E0640E751E808189831BC1F7
:1015C000043421F0043611F00936B1F5043411F475
:1015D00051E0552A50FE0AC0F30184E090E0680E05
:1015E000791E20813181428153810CC0F30142E098
:1015F00050E0640E751E808191819C01442737FD67
:101600004095542F2CA73DA74EA75FA78CA59DA55D
:10161000AEA5BFA5B7FF0DC0B095A09590958195DB
:101620009F4FAF4FBF4F8CA79DA7AEA7BFA78DE21F
:1016300089A77AE0472E7BC00F3411F00F3639F4BA
:101640000F3411F491E0592A68E0462E6FC000373C
:10165000A1F4F301A2E0B0E06A0E7B1E80819181CB
:101660009C01442755272CA73DA74EA75FA750E113
:10167000452E30E4532A08E759C00337C1F5F3017A
:1016800042E050E0640E751E8080918081149104C8
:1016900089F44E010894811C911C88E289838EE6AE
:1016A000F401818385E78B838CE68C838D8389E2CB
:1016B0008E831F8217FD13C0812F992787FD909578
:1016C000AC0160E070E0C4010E943B42009729F049
:1016D000D82ED8181D150CF090C0D12E8EC0F40154
:1016E00001900020E9F73197DE2ED81886C0053525
:1016F00011F0053739F4053511F4F1E05F2A4AE0BD
:10170000442E14C0083519F0083709F06CC030E1D8
:10171000432E53FE0BC02CA53DA54EA55FA521155C
:1017200031054105510511F030E4532A19A618ABD3
:1017300017FD02C04FED542229E2822E912C8C0E0F
:101740009D1E8CA59DA5AEA5BFA50097A105B105C1
:1017500021F498A9992309F43FC0C42CDD24EE2478
:10176000FF2433242CA53DA54EA55FA52C153D05D2
:101770004E055F0510F091E0392E6CA57DA58EA574
:101780009FA5A70196010E940244DC01CB01182FFE
:101790008A3010F4105D04C0195A083509F41F7D11
:1017A000D4011E934D016CA57DA58EA59FA5A70113
:1017B00096010E9402442CA73DA74EA75FA73320A5
:1017C00081F6B8E04B1641F453FE06C0103321F009
:1017D00080E3F40182934F01CE010196D82ED818F0
:1017E000F8E2DF0E0BC0002309F44EC04E0108944E
:1017F000811C911C098381E0D82E19A61D2DC8A833
:10180000CD18C7FCCC2489A5882311F01F5F02C026
:1018100056FC1E5F1C0DE52CFF24C70180739070E1
:10182000892B21F4822D811B0E94BB0989A5882365
:1018300029F061E070E0CE01899609C0E6FE09C09A
:1018400080E38AA70BA762E070E0CE018A960E942F
:101850009209C70180739070809721F4822D811BBB
:101860000E94C7098C2D0E94C7098D2D992787FDDD
:101870009095BC01C4010E949209E4FEC1CD822D65
:10188000811B0E94BB09BCCDE0960FB6F894DEBF69
:101890000FBECDBFDF91CF911F910F91FF90EF90C1
:1018A000DF90CF90BF90AF909F908F907F906F9080
:1018B0005F904F903F902F9008951F920F920FB618
:1018C0000F9211242F933F935F936F937F938F9386
:1018D0009F93AF93BF93EF93FF938091CC038823A3
:1018E00029F08091CC0381508093CC038091D40364
:1018F00081508093D4038F3FB9F489E08093D4035F
:1019000080910A038F5F817080930A03882319F402
:1019100081E08093D1038091D2039091D30301960B
:101920009093D3038093D2038091CD039091CE0303
:101930000297C8F08091CD039091CE0301979093C8
:10194000CE038093CD038091CD039091CE0320915F
:1019500006033091070382239323892B11F021E0A2
:1019600009C020E007C020E08FEF9FEF90930703AE
:101970008093060380910101222331F08A3011F413
:101980005A9A07C0479A05C08A3011F45A9801C084
:10199000479880916D0783FF5EC086B19927FC014F
:1019A000E071F07084FF0AC08091CF039091D00362
:1019B00001969093D0038093CF034DC08091CF03C5
:1019C0009091D003892B69F18091CF039091D0033E
:1019D0008A56914030F58091CF039091D00369E20F
:1019E00070E00E94DB438091CF039091D003860F7B
:1019F000971F9093D0038093CF038091CF03909152
:101A0000D0030B9750F08091CF039091D0030A97A9
:101A1000909341048093400404C0F0934104E09308
:101A20004004809140049091410420913E04309103
:101A30003F04821B930B845E9D4F68E671E00E9419
:101A4000EF43845B904090933D0480933C0410925C
:101A5000D0031092CF03FF91EF91BF91AF919F916F
:101A60008F917F916F915F913F912F910F900FBE5A
:101A70000F901F9018952091D2033091D303280F17
:101A8000391FC901019608958AE090E00E943B0D3C
:101A90009093D6038093D50382E085BD83EA84BD0D
:101AA00017BC88E788BD86E086BD83EC8093B000D4
:101AB00084E08093B1008091700082608093700018
:101AC00080916E00816080936E008AE08093B30005
:101AD0001092B20008952091D2033091D303821B5B
:101AE000930B892F99278695807490700895CF93D2
:101AF000DF930E943B0DEC01CE010E946B0D882309
:101B0000D9F3DF91CF910895CF93DF930E943B0DDE
:101B1000EC0103C08FEE80937A00CE010E946B0D22
:101B20008823C1F3DF91CF9108951F920F920FB6D2
:101B30000F9211248F939F93809108039091090332
:101B4000892B11F05F9A01C05F9883E08093B00009
:101B5000809170008E7F809370009F918F910F9085
:101B60000FBE0F901F9018951F920F920FB60F92F5
:101B700011242F933F934F935F936F937F938F9392
:101B80009F93AF93BF93CF93DF93EF93FF93809196
:101B9000080390910903049709F0A6C080E390E040
:101BA0009093CB038093CA0380910C0390910D0313
:101BB0009C01220F331F280F391F8091760399272C
:101BC000880F991F280F391F37FF02C02D5F3F4F25
:101BD000C901959587959595879590930D03809369
:101BE0000C03EC01E096D093CB03C093CA03809121
:101BF0009A079091870720917A0430917B04409155
:101C00007C0450917D0480FF18C0892F9927AA2752
:101C1000BB27BC01CD010E94B04397FF04C06150B7
:101C2000704C8F4F9F4F5EE09595879577956795A0
:101C30005A95D1F7C60FD71F17C0892F9927AA2702
:101C4000BB27BC01CD010E94B04397FF04C0615087
:101C5000704C8F4F9F4F4EE0959587957795679580
:101C60004A95D1F7C61BD70BD093CB03C093CA03B9
:101C70008091880743E0849FC00111242091CA030A
:101C80003091CB032817390740F080918907849F52
:101C9000C00111248217930720F49093CB03809303
:101CA000CA032091CA033091CB03309306072093D7
:101CB0000507C9016FEF70E00E94DB438D9740F488
:101CC000235B3F4F3093CB032093CA0383E101C0D2
:101CD00080E680930B038091CA039091CB0380959B
:101CE0008093B30083EC40C0809108039091090376
:101CF000892B39F18091080390910903049708F525
:101D00002091CA033091CB032F3F310561F058F089
:101D10005F9A83E08093B0002F5F30403093CB0315
:101D20002093CA0323C083E88093B00080910B0303
:101D30008093B30081E090E09093090380930803BF
:101D400015C08091080390910903892B79F4809143
:101D50008A079927880F991F880F991F9093090365
:101D6000809308035F9883E08093B000809108031C
:101D70009091090301979093090380930803FF91C1
:101D8000EF91DF91CF91BF91AF919F918F917F9113
:101D90006F915F914F913F912F910F900FBE0F90D8
:101DA0001F90189510927C008FEE80937A00089512
:101DB0000F931F93CF93DF9303E010E0D8010E94AD
:101DC0003F44802DC82FDD27C531D10508F02A9763
:101DD000C7BD84E690E00E94840D80910E0390912F
:101DE0000F038255934010F4C0E0D0E0CA3FD10504
:101DF000C0F4C7BD82E390E00E94840D80E791E0CB
:101E00009F938F931F920E94D30980910E0390910C
:101E10000F030F900F900F908458934010F021966D
:101E2000E5CFD8010C2E0E944744C0932C078CE2CA
:101E300091E00E94840DDF91CF911F910F91089541
:101E40001F920F920FB60F921124EF92FF920F93F1
:101E50001F932F933F934F935F936F937F938F9332
:101E60009F93AF93BF93CF93DF93EF93FF93109222
:101E70007A008091EE03682F77278F5F8093EE03BF
:101E80006530710509F48EC066307105BCF46230AE
:101E9000710509F44AC0633071053CF461157105A0
:101EA00031F161307105C1F1AEC26330710509F4E1
:101EB00046C06430710509F45DC0A5C26830710583
:101EC00009F4C3C0693071054CF46630710509F43A
:101ED00082C06730710509F49BC095C269307105F5
:101EE00009F4D0C06A30710509F4EBC18CC280914D
:101EF0007800909179009093F0038093EF0381E054
:101F00008093ED038091D7039091D803019690932D
:101F1000D8038093D7037BC2809178009091790099
:101F20009093F2038093F1038EC08091780090919A
:101F300079009093F4038093F30384E0BFC1809110
:101F40001403909115039C01220F331F280F391F92
:101F500080917800909179000E94DB43260F371F13
:101F600036952795369527953093150320931403BE
:101F700086E0A4C180918604909187042091780026
:101F800030917900821B930B9093200780931F0759
:101F900080911F07909120079093E6038093E503BB
:101FA00087E08CC18091780090917900209188041D
:101FB00030918904821B930B90932B0780932A07FF
:101FC00080912A0790912B079093E4038093E30379
:101FD0001092ED031CC2809101012091EF0330911A
:101FE000F0038A3049F48091780090917900820F53
:101FF000931F9695879506C08091780090917900FF
:10200000820F931F9093E8038093E70381E056C10A
:10201000809101012091F1033091F2038A3049F45B
:102020008091780090917900820F931F9695879503
:1020300006C08091780090917900820F931F909351
:10204000EA038093E90382E039C180910101209184
:10205000F3033091F4038A3049F480917800909131
:102060007900820F931F9695879506C0809178001E
:1020700090917900820F931F9093EC038093EB0370
:1020800085E01CC18091780090917900AA2797FD86
:10209000A095BA2FBC01CD010E94EE427B018C01BC
:1020A0008091800490918104A0918204B091830476
:1020B0009C01AD01C801B7010E944842DC01CB017F
:1020C000BC01CD010E94D142DC01CB019093E2031F
:1020D0008093E1038091E1039091E20302970CF475
:1020E00046C08091800490918104A0918204B091B7
:1020F000830420E030E84BE354E4BC01CD010E94AE
:10210000F84288230CF088C080918004909181046B
:10211000A0918204B09183042AE037ED43EA5CE3A6
:10212000BC01CD010E944942DC01CB0180938004B7
:1021300090938104A0938204B0938304809101045E
:1021400090910204845F914008F066C08091800401
:1021500090918104A0918204B09183042DEC3CEC19
:102160004CEC5DE3BC01CD010E9449424BC0809123
:10217000E1039091E2038F5F9F4F0CF04DC080917F
:10218000800490918104A0918204B091830420E0A6
:1021900030E849E054E4BC01CD010E94FB4218162E
:1021A000DCF58091800490918104A0918204B0912B
:1021B00083042AE037ED43EA5CE3BC01CD010E94D1
:1021C0004842DC01CB018093800490938104A0936A
:1021D0008204B09383048091010490910204845F8F
:1021E0009140D0F48091800490918104A091820468
:1021F000B09183042DEC3CEC4CEC5DE3BC01CD01D3
:102200000E944842DC01CB018093800490938104BA
:10221000A0938204B093830481E08093DB038091D8
:102220007800909179009093220780932107809104
:10223000E1039091E2039C01442737FD4095542F20
:102240008091420490914304A0914404B0914504CC
:10225000820F931FA41FB51F8093420490934304E1
:10226000A0934404B0934504209142043091430468
:10227000409144045091450457FF04C021503C4F05
:102280004F4F5F4FAAE05595479537952795AA95EB
:10229000D1F78091420490914304A0914404B091FD
:1022A0004504821B930BA40BB50B809342049093BF
:1022B0004304A0934404B093450483E08093ED036A
:1022C000A6C080912F07909130072091780030911F
:1022D0007900820F931F9093300780932F0780918E
:1022E00027078F5F8093270780912707853008F4A1
:1022F0008AC0809178009091790090930F03809329
:102300000E03109227078091D9039091DA03BC0144
:10231000F3E0660F771FFA95E1F7681B790B809160
:102320007F03482F55278091230790912407209100
:102330002F0730913007821B930B2091230430919B
:102340002404821B930B489F9001499F300D589F96
:10235000300D1124620F731F77FF02C0695F7F4F3A
:10236000E3E075956795EA95E1F77093DA0360937A
:10237000D90380912F0790913007EC01EE27D7FD0C
:10238000E095FE2F2091100330911103409112032C
:1023900050911303DA01C901880F991FAA1FBB1FAF
:1023A000820F931FA41FB51FC80FD91FEA1FFB1F61
:1023B000F7FF03C02396E11DF11D82E0F595E79537
:1023C000D795C7958A95D1F7C0931003D093110381
:1023D000E0931203F0931303809110039091110383
:1023E000A0911203B09113039C0180912307909157
:1023F0002407821B930B9093240480932304109250
:10240000300710922F071092ED031092EE03809187
:10241000ED0380937C008091EE03882319F08FEE0A
:1024200080937A00FF91EF91DF91CF91BF91AF91AF
:102430009F918F917F916F915F914F913F912F91DC
:102440001F910F91FF90EF900F900FBE0F901F9074
:10245000189590E2E6E1F3E08FE49193815087FFD5
:10246000FCCF08951F93CF93DF938091F50380FFF6
:102470000FC08091F903882311F0815002C0809130
:1024800070038093F9030E9429128FEF8093B703A2
:102490008091F50381FF0AC08091F9038F5F8093DB
:1024A000F9030E9429128FEF8093B7038091F503FF
:1024B000992780FF04C081FF02C01092F903809128
:1024C000F903282F33278A3040F481E18093F60303
:1024D0003F932F9382E791E007C080E18093F6035A
:1024E0003F932F9387E791E09F938F9381E08F93A2
:1024F0000E94D3090F900F900F900F900F90809132
:10250000F903C82FDD27C530D10509F46AC2C630EA
:10251000D105ACF4C230D10509F4E9C0C330D1050E
:1025200034F4209739F1219709F477C0FDC4C33002
:10253000D10509F44EC1249709F4B7C1F5C4C830D8
:10254000D10509F4A9C3C930D10544F4C630D10579
:1025500009F41CC3279709F47EC3E6C4CA30D10529
:1025600009F432C4CA30D1050CF4D9C32B9709F44D
:1025700071C4DAC41092F6038CE791E09F938F93B5
:1025800011E01F930E94D30984E18093F6030F901A
:102590000F900F908CE690E09F938F9385E490E0EE
:1025A0009F938F93DF93CF93809101016AE00E9404
:1025B000CF43892F99279F938F93809101010E9488
:1025C000CF4399279F938F938CE891E09F938F93AC
:1025D0001F930E94D30988E28093F6038DB79EB7BC
:1025E0000D960FB6F8949EBF0FBE8DBF0E94790264
:1025F00099279F938F9381EA91E09F938F931F93E5
:102600000E94D3098CE38093F6030F900F900F90F4
:102610000F900F908EEA91E061C080916D0780FF6E
:102620004AC01092F60380912304909124049F9352
:102630008F938EEB91E09F938F9311E01F930E94F5
:10264000D30984E18093F6030F900F900F900F90C1
:102650000F9080912104909122049F938F938DEC91
:1026600091E09F938F931F930E94D30988E28093F8
:10267000F6030F900F900F900F900F9080910E0324
:1026800090910F039F938F938CED91E09F938F9385
:102690001F930E94D3098CE38093F6030F900F9051
:1026A0000F900F900F9080912C0799279F938F93F5
:1026B0008BEE91E07EC384E18093F6038AEF91E094
:1026C0009F938F9311E01F930E94D30988E2809318
:1026D000F6030F900F900F9081E092E09F938F93FD
:1026E0001F930E94D3090F900F900F9022C4109255
:1026F000F6038FE092E09F938F93C1E0CF930E9407
:10270000D30984E18093F6030F900F900F9080918E
:102710007A0490917B04A0917C04B0917D04B7FF72
:1027200004C081509C4FAF4FBF4F6AE0B595A7954D
:10273000979587956A95D1F7BF93AF939F938F93A2
:1027400089E192E09F938F93CF930E94D30988E20F
:102750008093F6038DB79EB707960FB6F8949EBF89
:102760000FBE8DBF8091720490917304A091740488
:10277000B0917504B7FF04C081509C4FAF4FBF4F5D
:102780005AE0B595A795979587955A95D1F7BF9338
:10279000AF939F938F9388E292E09F938F93CF9311
:1027A0000E94D3098CE38093F6038DB79EB70796FA
:1027B0000FB6F8949EBF0FBE8DBF809140049091DC
:1027C00041049F938F9387E392E09F938F93CF93DE
:1027D000F3C21092F60380913D0790913E079F93BC
:1027E0008F9380913B0790913C079F938F9386E452
:1027F00092E09F938F9311E01F930E94D30984E18D
:102800008093F6038DB79EB707960FB6F8949EBFD8
:102810000FBE8DBF80914107909142079F938F9388
:1028200080913F07909140079F938F9386E592E0B8
:102830009F938F931F930E94D30988E28093F6039E
:102840008DB79EB707960FB6F8949EBF0FBE8DBF8B
:1028500080914507909146079F938F9380914307FE
:10286000909144079F938F9386E692E09F938F9376
:102870001F930E94D3098CE38093F6038DB79EB714
:1028800007960FB6F8949EBF0FBE8DBF8091490783
:1028900090914A079F938F938091470790914807A3
:1028A0009F938F9386E792E031C31092F603809155
:1028B0006607E82FFF27EE0FFF1FE75CF84F8081C8
:1028C00091819F938F9380916507E82FFF27EE0FEB
:1028D000FF1FE75CF84F808191819F938F9386E87B
:1028E00092E09F938F9311E01F930E94D30984E19C
:1028F0008093F6038DB79EB707960FB6F8949EBFE8
:102900000FBE8DBF80916807E82FFF27EE0FFF1FD6
:10291000E75CF84F808191819F938F938091670747
:10292000E82FFF27EE0FFF1FE75CF84F80819181B2
:102930009F938F9386E992E09F938F931F930E94BA
:10294000D30988E28093F6038DB79EB707960FB63A
:10295000F8949EBF0FBE8DBF80916A07E82FFF27B6
:10296000EE0FFF1FE75CF84F808191819F938F935B
:1029700080916907E82FFF27EE0FFF1FE75CF84FF4
:10298000808191819F938F9386EA92E09F938F93AA
:102990001F930E94D3098CE38093F6038DB79EB7F3
:1029A00007960FB6F8949EBF0FBE8DBF80916C073F
:1029B000E82FFF27EE0FFF1FE75CF84F8081918122
:1029C0009F938F9380916B07E82FFF27EE0FFF1FD8
:1029D000E75CF84F808191819F938F9386EB92E023
:1029E00095C21092F60386EC92E09F938F93C1E01C
:1029F000CF930E94D309809101010F900F900F9007
:102A00008A3009F05AC084E18093F60380919204E1
:102A1000909193049F938F938091EB039091EC039B
:102A20002091920430919304821B930B9F938F9378
:102A300084ED92E09F938F93CF930E94D30988E215
:102A40008093F6038DB79EB707960FB6F8949EBF96
:102A50000FBE8DBF80919004909191049F938F93AE
:102A60008091E9039091EA032091900430919104C0
:102A7000821B930B9F938F9383EE92E09F938F9390
:102A8000CF930E94D3098CE38093F6038DB79EB752
:102A900007960FB6F8949EBF0FBE8DBF80918E042F
:102AA00090918F049F938F938091D8079091D9072D
:102AB0009F938F9382EF92E065C084E18093F60349
:102AC000809192049091930497FD01969595879536
:102AD0009F938F938091EB039091EC03209192044C
:102AE00030919304821B930B9F938F9381E093E02B
:102AF0009F938F93CF930E94D30988E28093F6032C
:102B00008DB79EB707960FB6F8949EBF0FBE8DBFC8
:102B1000809190049091910497FD019695958795E9
:102B20009F938F938091E9039091EA032091900401
:102B300030919104821B930B9F938F9380E193E0DC
:102B40009F938F93CF930E94D3098CE38093F603D6
:102B50008DB79EB707960FB6F8949EBF0FBE8DBF78
:102B600080918E0490918F0497FD0196959587959D
:102B70009F938F938091D8079091D9079F938F93BC
:102B80008FE193E09F938F93CF93C3C11092F6038D
:102B90008EE293E09F938F9311E01F930E94D309DD
:102BA00084E18093F6030F900F900F90809188043A
:102BB000909189049F938F938091E3039091E40314
:102BC0009F938F938BE393E09F938F931F930E9428
:102BD000D30988E28093F6038DB79EB707960FB6A8
:102BE000F8949EBF0FBE8DBF80918604909187049C
:102BF0009F938F938091E5039091E6039F938F932A
:102C00008AE493E09F938F931F930E94D3098CE3F0
:102C10008093F6038DB79EB707960FB6F8949EBFC4
:102C20000FBE8DBF8091800490918104A091820499
:102C3000B0918304BC01CD010E94D142DC01CB01E3
:102C40009F938F938091BE079091BF079F938F931F
:102C500089E593E05BC184E18093F60380911403DE
:102C6000909115039F938F9388E693E09F938F93A2
:102C700011E01F930E94D30988E28093F6030F901E
:102C80000F900F900F900F9080912E0499279F9393
:102C90008F9387E793E08DC01092F60386E893E068
:102CA0009F938F9311E01F930E94D30984E1809337
:102CB000F6030F900F900F9080913C0490913D048B
:102CC0009F938F9385E993E09F938F931F930E9427
:102CD000D30988E28093F6030F900F900F900F9026
:102CE0000F9080914004909141049F938F9384EAC8
:102CF00093E09F938F931F930E94D3098CE380935B
:102D0000F6030F900F900F900F900F9080913E045C
:102D100090913F049F938F9383EB93E04AC010926E
:102D2000F60380913504909136049F938F9382EC43
:102D300093E09F938F9311E01F930E94D30984E146
:102D40008093F6030F900F900F900F900F9080914B
:102D50003304909134049F938F938EEC93E09F9370
:102D60008F931F930E94D30988E28093F6030F90FC
:102D70000F900F900F900F9080913104909132043A
:102D80009F938F938AED93E09F938F931F930E945D
:102D9000D3098CE38093F6030F900F900F900F9060
:102DA0000F9080912F04909130049F938F9386EE23
:102DB00093E09F938F931F930E94D3090F900F90DE
:102DC0000F900F900F90B5C01092F60382EF93E032
:102DD0009F938F9311E01F930E94D30984E1809306
:102DE000F6030F900F900F908091760399279F9391
:102DF0008F938AEF93E09F938F931F930E94D30941
:102E000088E28093F6030F900F900F900F900F9031
:102E10008091CA039091CB039F938F9388E094E0B5
:102E20009F938F931F930E94D3098CE38093F603A3
:102E30000F900F900F900F900F9080918907992716
:102E40009F938F938091880799279F938F9386E113
:102E500094E05CC01092F60384E294E09F938F9319
:102E600011E01F930E94D30984E18093F6030F9031
:102E70000F900F9080913C06992787FD90959F9326
:102E80008F9380913B06992787FD90959F938F9311
:102E900084E394E09F938F931F930E94D30988E269
:102EA0008093F6038DB79EB707960FB6F8949EBF32
:102EB0000FBE8DBF80913D06992787FD90959F930A
:102EC0008F9380913E0699279F938F9384E494E09B
:102ED0009F938F931F930E94D3098CE38093F603F3
:102EE0008DB79EB707960FB6F8949EBF0FBE8DBFE5
:102EF0008091420699279F938F9380913F0699274F
:102F000087FD90959F938F9384E594E09F938F9393
:102F10001F930E94D3098DB79EB707960FB6F894FA
:102F20009EBF0FBE8DBF05C081508093700310926D
:102F3000F9031092F503DF91CF911F91089510923C
:102F4000B9008AE28093B800089585EA8093BC00B6
:102F500080E090E0089584E98093BC000895109289
:102F6000B9008093BB0085E88093BC0080E090E0CE
:102F700008950E94AB171092FC038091BB00109241
:102F8000FB0380E88093BC001092BD001092BA0051
:102F90001092BB001092B9001092B8000E949F17C7
:102FA0000E94A51780E00E94AF1708951F920F920C
:102FB0000FB60F9211242F933F934F935F936F930C
:102FC0007F938F939F93AF93BF93EF93FF938091E2
:102FD000FC03282F33278F5F8093FC0323303105B8
:102FE00009F446C0243031054CF421303105D1F0CC
:102FF000223031057CF5232B81F083C0253031054B
:10300000E1F1253031050CF441C026303105F1F1F4
:103010002730310509F45AC074C08091FB03880F32
:103020008E5A51C08091FB03282F33278F5F8093E6
:10303000FB032130310509F43EC0223031051CF478
:10304000232BB1F15EC022303105C1F123303105AF
:10305000C1F157C00E94AB178091FB03843018F474
:103060001092FC0302C01092FB030E94A51749C0F6
:103070008091FA03880F8D5A26C08091FA03E82FB9
:10308000FF27EF5CF84F8091BB0080838091FA03AB
:1030900099278130910579F0823091051CF4892BB4
:1030A00039F02FC08230910549F0039751F029C0C3
:1030B0008091AF0708C08091B60705C08091D00706
:1030C00002C08091D2070E94AF171BC09091FA03F3
:1030D000E92FFF27EF5CF84F8091BB008483892F95
:1030E0008F5F8093FA03843010F01092FA030E94ED
:1030F000AB178AE090E090938F0380938E03109239
:10310000FC038091BC0080688093BC00FF91EF912C
:10311000BF91AF919F918F917F916F915F914F91EF
:103120003F912F910F900FBE0F901F90189583EC39
:103130008093810080916F00806280936F00109275
:103140008F0410928E0410929104109290041092A9
:1031500093041092920408951F920F920FB60F924B
:1031600011240F931F932F933F934F935F936F936C
:103170007F938F939F93AF93BF93CF93DF93EF93FF
:10318000FF9340918600509187008091FD039091BC
:10319000FE03481B590B8091860090918700909305
:1031A000FE038093FD03CA018D549440A091FF0358
:1031B000B0910004835F9A4158F4149714F0109270
:1031C000710381E090E0909300048093FF0399C025
:1031D000AA30B1050CF095C0CA018B5F9040845BAA
:1031E000914008F071C0425D5140FD01EA0FFB1FA4
:1031F000E75CF84F80819181FA01E81BF90BCF0160
:10320000F7FF03C0909581959F4F06974CF48091EE
:103210002E04883C28F480912E04865F80932E042F
:10322000FD01EA0FFB1FE75CF84F808191819C0153
:10323000220F331F280F391F240F351F37FF02C0FD
:103240002D5F3F4FE901D595C795D595C795CA0123
:1032500001968C179D0714F4219706C041505040E9
:10326000C417D5070CF4219680912E04833CD8F026
:103270008D010A0F1B1FF801E75CF84F80819181D7
:103280009E01281B390BC90163E070E00E94EF43E7
:10329000CB01880F991F860F971F015B184FF8010C
:1032A0009183808307C0AA0FBB1FA15BB84F119603
:1032B0001C921E92E091FF03F0910004EE0FFF1F9D
:1032C000E75CF84FD183C0838091FF0390910004A5
:1032D0000196909300048093FF03059711F45D9A83
:1032E00001C05D988091FF039091000486309105A4
:1032F00011F45C9A01C05C98079711F45B9A01C0C5
:103300005B98FF91EF91DF91CF91BF91AF919F912A
:103310008F917F916F915F914F913F912F911F916D
:103320000F910F900FBE0F901F90189581E0809322
:10333000650782E08093660783E08093670754E027
:103340005093680735E03093690786E080936A07F9
:1033500087E080936B0728E020936C0788E68093D2
:103360006D079EE190936E078BEF809370078AE064
:103370008093710790936F07909373075093720730
:103380008FE080937407909375076CE060937607E5
:103390002093770786EE809378079093790780E8EB
:1033A00080937A0780E580937B0746E940937C070A
:1033B0008EE580937D0783E280937E0790937F075D
:1033C0001092800780E2809381078DEF80938207BF
:1033D00024E6209383079AE59093840790938507CA
:1033E00090939507909396071092970710929807DD
:1033F0002093860788E28093870710929A0782E3DA
:10340000809388074093890730938A0780938B07BE
:1034100090938C0780938D071092990790938E0755
:1034200030938F07209390072093910780E180933A
:1034300092075093930720939407AFE9B7E0E0E930
:10344000F3E001900D926150E1F7089581E08093DF
:10345000650782E08093660743E04093670774E066
:103460007093680755E05093690736E030936A0718
:1034700087E080936B0728E020936C0788E68093B1
:103480006D079EE190936E078BEF809370078AE043
:103490008093710790936F0790937307409372071F
:1034A0006CE06093740780E1809375073093760732
:1034B0002093770786EE809378079093790780E8CA
:1034C00080937A0780E580937B0788E780937C0769
:1034D0008EE580937D0783E280937E0790937F073C
:1034E0001092800740E2409381078DEF809382071E
:1034F00034E6309383072AE52093840720938507D9
:10350000209395072093960710929707109298079B
:103510003093860788E28093870710929A0792E398
:103520009093880786E98093890750938A07909340
:103530008B0720938C0790938D0710929907209307
:103540008E0750938F0730939007309391074093E5
:103550009207709393078BE480939407AFE9B7E0E9
:10356000E7E9F3E001900D926150E1F7089581E001
:103570008093650782E08093660743E04093670786
:1035800064E06093680755E05093690736E0309334
:103590006A0787E080936B0728E020936C0788EE2A
:1035A00080936D079EE190936E078BEF8093700779
:1035B0008AE08093710790936F079093730740930D
:1035C00072072093740740E14093750730937607A4
:1035D0002093770786EE809378079093790780E8A9
:1035E00080937A0734E630937B0788E780937C07E3
:1035F0008EE580937D0783E280937E0784E180934C
:103600007F0710928007409381078DEF8093820798
:10361000309383079AE5909384079093850790935E
:1036200095079093960710929707109298073093FA
:10363000860788E28093870710929A0722E32093F7
:10364000880786E98093890750938A0720938B0720
:1036500090938C0720938D071092990790938E0773
:1036600050938F07309390073093910780E28093B7
:1036700092076093930720939407AFE9B7E0EFE9CF
:10368000F3E08CE001900D928150E1F70895CF9323
:10369000C82FC150CF3F81F080912504882361F469
:1036A00084E690E09093CE038093CD038AEF90E080
:1036B0000E94770DC15080F7CF91089510927A0043
:1036C0008091EB039091EC039093B8078093B70738
:1036D0008091E9039091EA039093AE078093AD0740
:1036E0008091E7039091E8039093D9078093D807DE
:1036F0008091E3039091E403AA2797FDA095BA2F48
:10370000BC01CD012CE030E040E050E00E94B0432D
:10371000DC01CB019093D6078093D5078091E50318
:103720009091E603AA2797FDA095BA2FBC01CD0181
:103730000E94B043DC01CB019093E6078093E5073C
:103740008091E1039091E2039093BF078093BE07BD
:103750008FEE80937A0080916907E82FFF27EE0FA4
:10376000FF1FE75CF84F8081918182599F4F209124
:10377000350430913604281739071CF42F5F3F4F6A
:103780000CC08081918182599F4F821793074CF41E
:103790002115310531F0215030403093360420930B
:1037A000350480916A07E82FFF27EE0FFF1FE75CC3
:1037B000F84F8081918182599F4F2091330430913D
:1037C0003404281739071CF42F5F3F4F0CC0808149
:1037D000918182599F4F821793074CF4211531052F
:1037E00031F02150304030933404209333048091E1
:1037F0006B07E82FFF27EE0FFF1FE75CF84F808174
:10380000918182599F4F20913104309132042817C1
:1038100039071CF42F5F3F4F0CC080819181825982
:103820009F4F821793074CF42115310531F0215039
:103830003040309332042093310480916C07E82F9C
:10384000FF27EE0FFF1FE75CF84F808191818259BF
:103850009F4F20912F0430913004281739071CF412
:103860002F5F3F4F0CC08081918182599F4F8217FB
:1038700093074CF42115310531F02150304030933D
:10388000300420932F04809135049091360497FFE3
:1038900005C010923604109235040AC08F3F91057E
:1038A00039F034F08FEF90E0909336048093350434
:1038B000809133049091340497FF05C01092340432
:1038C000109233040AC08F3F910539F034F08FEF26
:1038D00090E090933404809333048091310490916C
:1038E000320497FF05C010923204109231040AC0CE
:1038F0008F3F910539F034F08FEF90E090933204D0
:103900008093310480912F049091300497FF05C07B
:103910001092300410922F040AC08F3F910539F0A5
:1039200034F08FEF90E09093300480932F048091D7
:1039300090079927AA27BB27BC01CD0124EC39E0C9
:1039400040E050E00E94B043DC01CB01809388034B
:1039500090938903A0938A03B0938B03809191077E
:103960009927AA27BB27BC01CD010E94B043DC01E7
:10397000CB018093840390938503A0938603B09337
:103980008703089510928904109288041092870486
:103990001092860480E090E0A0E0B0E08093800484
:1039A00090938104A0938204B093830410929304B3
:1039B00010929204109291041092900410928F042D
:1039C00010928E0410920E0410920D040E945E1B41
:1039D00084E690E00E94840D0E945E1B80916D073A
:1039E00080FF10C080910E0390910F03875B93407E
:1039F00038F480910E0390910F038E5E924010F484
:103A00000E94D80E8091EB039091EC039093930465
:103A1000809392048091E9039091EA03909391043A
:103A2000809390048091E7039091E80390938F0432
:103A300080938E04809190049091910490938D04D2
:103A400080938C04809192049091930490938B04C2
:103A500080938A0444E050E0DA010E943F44802DC4
:103A6000853078F18091E5079091E6078091E50730
:103A70009091E60797FF03C0909581959F4F6CE06A
:103A800070E00E94EF4370938704609386048091F6
:103A9000D5079091D6078091D5079091D60797FFCB
:103AA00003C0909581959F4F6CE070E00E94EF43BA
:103AB0007093890460938804809121079091220774
:103AC00034C0DA010E943F44802D9927982F88271F
:103AD000DA0111960E943F44202D820F911D909390
:103AE000890480938804DA0112960E943F44802D55
:103AF0009927982F8827DA0113960E943F44202D9A
:103B0000820F911D9093870480938604DA011496A6
:103B10000E943F44802D9927982F8827DA01159617
:103B20000E943F44202D820F911DAA2797FDA0954A
:103B3000BA2FBC01CD010E94EE42DC01CB01809383
:103B4000800490938104A0938204B0938304109224
:103B50005A0410925B0410925C0410925D0410925F
:103B6000560410925704109258041092590410925F
:103B7000520410925304109254041092550410925F
:103B80004E0410924F04109250041092510410925F
:103B90004A0410924B0410924C0410924D0410925F
:103BA000B8071092B7071092AE071092AD071092A7
:103BB000D9071092D8078091100390911103A0911A
:103BC0001203B0911303909324078093230710925C
:103BD000DA031092D9031092420410924304109217
:103BE00044041092450480914004909141049093C4
:103BF0003F0480933E040E949D3F82E390E09093B7
:103C0000CE038093CD03809190079927AA27BB27E5
:103C1000BC01CD0124EC39E040E050E00E94B0430B
:103C2000DC01CB018856954CAF4FBF4F8093880382
:103C300090938903A0938A03B0938B03809191079B
:103C40009927AA27BB27BC01CD010E94B043DC0104
:103C5000CB018856954CAF4FBF4F80938403909310
:103C60008503A0938603B093870310927303109289
:103C700072038091400490914104AA2797FDA0957A
:103C8000BA2FBC01CD012EE036E040E050E00E94AA
:103C9000B043DC01CB018093E1079093E207A0934E
:103CA000E307B093E407109238041092370481E0E0
:103CB0008093000108959F92AF92BF92CF92DF92BE
:103CC000EF92FF920F931F93CF93DF9380918E0417
:103CD00090918F042091E7033091E803821B930BAE
:103CE0009093D9078093D8078091E9039091EA03D4
:103CF0002091900430919104821B930B9093AE0716
:103D00008093AD078091EB039091EC032091920496
:103D100030919304821B930B9093B8078093B7075D
:103D20008091AD079091AE07909316078093150789
:103D30008091D5079091D6077C010027F7FC00956C
:103D4000102F8091E3039091E403AA2797FDA0959B
:103D5000BA2FBC01CD012CE030E040E050E00E94E1
:103D6000B043DC01CB01E80EF91E0A1F1B1F17FF31
:103D700005C00894E11CF11C011D111D1595079546
:103D8000F794E794F092D607E092D5078091E50783
:103D90009091E6077C010027F7FC0095102F809199
:103DA000E5039091E603AA2797FDA095BA2FBC01E1
:103DB000CD012CE030E040E050E00E94B043DC0157
:103DC000CB01E80EF91E0A1F1B1F17FF05C0089440
:103DD000E11CF11C011D111D15950795F794E79441
:103DE000F092E607E092E5078091BE079091BF0749
:103DF0009C01442737FD4095542F8091E103909119
:103E0000E203AA2797FDA095BA2F280F391F4A1F52
:103E10005B1F57FF04C02F5F3F4F4F4F5F4F5595BC
:103E20004795379527953093BF072093BE0780911C
:103E3000E3039091E4036CE070E0869F9001879F1C
:103E4000300D969F300D1124C9019C01442737FD88
:103E50004095542F80916A0490916B04A0916C045A
:103E6000B0916D04820F931FA41FB51F80936A0445
:103E700090936B04A0936C04B0936D048091E50360
:103E80009091E603869F9001879F300D969F300D9D
:103E90001124C9019C01442737FD4095542F80917E
:103EA000660490916704A0916804B0916904820F40
:103EB000931FA41FB51F8093660490936704A0937B
:103EC0006804B09369048091C6079091C707209158
:103ED000E3033091E403820F931F9093C70780930D
:103EE000C6078091DA079091DB072091E5033091B6
:103EF000E603820F931F9093DB078093DA0780918C
:103F000084049091850401969093850480938404A1
:103F10008091620490916304A0916404B09165045F
:103F2000BC01CD010E94EE425B016C018091210732
:103F300090912207AA2797FDA095BA2FBC01CD0129
:103F40000E94EE427B018C0180918004909181045B
:103F5000A0918204B09183049C01AD01C801B70116
:103F60000E944842DC01CB019C01AD01C601B501B4
:103F70000E944942DC01CB01BC01CD010E94D1422B
:103F8000DC01CB018093620490936304A0936404EA
:103F9000B09365048091D8079091D907AA2797FD1F
:103FA000A095BA2FC091E107D091E207E091E30715
:103FB000F091E407C80FD91FEA1FFB1FC093E10768
:103FC000D093E207E093E307F093E4078091D807EA
:103FD0009091D9079C01442737FD4095542F80913B
:103FE0004A0490914B04A0914C04B0914D04820F6F
:103FF000931FA41FB51F80934A0490934B04A09372
:104000004C04B0934D048091D8079091D9079C013E
:10401000442737FD4095542F8091460490914704E2
:10402000A0914804B0914904820F931FA41FB51FAB
:104030008093460490934704A0934804B0934904A6
:10404000C03B33E8D30738E0E30730E0F30764F020
:10405000C05BD348E840F040C093E107D093E2074B
:10406000E093E307F093E4078091E1079091E20782
:10407000A091E307B091E407B7FF0CC080559C47BF
:10408000A74FBF4F8093E1079093E207A093E30708
:10409000B093E40790901C04992009F0C3C080916C
:1040A0001B04882309F0BEC080916D0786FFBAC04B
:1040B0008091D8079091D907AA2797FDA095BA2F8C
:1040C00020915A0430915B0440915C0450915D044E
:1040D000BC01CD010E94B0439B01AC0197FF04C01D
:1040E0002150384F4F4F5F4F6BE0559547953795AF
:1040F00027956A95D1F780910E04E82EFF240027BA
:104100001127CA01B901A80197010E94B043DC013F
:10411000CB018093940490939504A0939604B0935C
:104120009704B7FF04C08150904FAF4FBF4F5C0161
:104130006D013CE0D594C794B794A7943A95D1F714
:10414000A0929404B0929504C0929604D0929704E1
:104150008091D8079091D907AA2797FDA095BA2FEB
:1041600020915204309153044091540450915504CD
:10417000BC01CD010E94B04397FF04C06150784F4D
:104180008F4F9F4F2BE095958795779567952A954B
:10419000D1F7A80197010E94B043DC01CB018093C5
:1041A000980490939904A0939A04B0939B04B7FF4A
:1041B00004C08150904FAF4FBF4F9C01AD011CE038
:1041C00055954795379527951A95D1F720939804DB
:1041D0003093990440939A0450939B04D601C501EF
:1041E000D7FE07C0B095A095909581959F4FAF4F92
:1041F000BF4F81389105A105B10584F4DA01C901E9
:1042000057FF07C0B095A095909581959F4FAF4FF0
:10421000BF4F81389105A105B105A4F081E08093DD
:10422000390410C0109298041092990410929A04C4
:1042300010929B041092940410929504109296048C
:10424000109297048091AD079091AE07209194044D
:1042500030919504820F931F9093AE078093AD0722
:1042600000910D04202F332744275527809198046F
:1042700090919904A0919A04B0919B04BC01CD0146
:104280000E94B0439B01AC0197FF04C021503E4FF8
:104290004F4F5F4FC9E05595479537952795CA957C
:1042A000D1F78091AD079091AE07820F931F909345
:1042B000AE078093AD078091AD079091AE079C014A
:1042C000442737FD4095542F80914E0490914F0420
:1042D000A0915004B0915104820F931FA41FB51FE9
:1042E00080934E0490934F04A0935004B0935104D4
:1042F0008091AD079091AE0720911F04309120046A
:10430000821B930B9C01442737FD4095542F8091CD
:10431000520490915304A0915404B0915504820F1B
:10432000931FA41FB51F8093520490935304A0932E
:104330005404B0935504C0918403D0918503E09157
:104340008603F0918703C817D907EA07FB07C4F46F
:1043500088EA91E6A0E0B0E08C1B9D0BAE0BBF0B92
:104360008093520490935304A0935404B093550443
:1043700080934E0490934F04A0935004B093510443
:1043800022273327A9012C1B3D0B4E0B5F0B80917D
:10439000520490915304A0915404B0915504821793
:1043A0009307A407B507B4F4CE01DF01885A9146FC
:1043B000A040B0408093520490935304A0935404BF
:1043C000B093550480934E0490934F04A0935004EF
:1043D000B09351048091E9039091EA030F9734F46C
:1043E00088E19CEF9093AE078093AD078091E9033D
:1043F0009091EA03079734F480E398EF9093AE0727
:104400008093AD07109101011A30A9F48091E9035E
:104410009091EA03835F934034F088EE93E09093A9
:10442000AE078093AD078091E9039091EA038A5F1C
:104430009340DCF014C08091E9039091EA03855E1B
:10444000974034F088EE93E09093AE078093AD07E9
:104450008091E9039091EA03835F974034F080ED07
:1044600097E09093AE078093AD078091B707909146
:10447000B8072091980430919904821B930B909374
:10448000B8078093B707202F3327442755278091FB
:10449000940490919504A0919604B0919704BC0166
:1044A000CD010E94B0439B01AC0197FF04C0215095
:1044B0003E4F4F4F5F4FB9E055954795379527953C
:1044C000BA95D1F78091B7079091B807821B930BEB
:1044D0009093B8078093B7078091B7079091B8077A
:1044E0009C01442737FD4095542F809156049091AC
:1044F0005704A0915804B0915904820F931FA41F30
:10450000B51F8093560490935704A0935804B0931A
:1045100059048091B7079091B80720911D043091FC
:104520001E04821B930B9C01442737FD4095542F9A
:1045300080915A0490915B04A0915C04B0915D0459
:10454000820F931FA41FB51F80935A0490935B049E
:10455000A0935C04B0935D04C0918803D09189035B
:10456000E0918A03F0918B03C817D907EA07FB078C
:10457000C4F488EA91E6A0E0B0E08C1B9D0BAE0B82
:10458000BF0B80935A0490935B04A0935C04B09398
:104590005D048093560490935704A0935804B093FD
:1045A000590422273327A9012C1B3D0B4E0B5F0B0F
:1045B00080915A0490915B04A0915C04B0915D04D9
:1045C00082179307A407B507B4F4CE01DF01885A18
:1045D0009146A040B04080935A0490935B04A0930E
:1045E0005C04B0935D048093560490935704A093A9
:1045F0005804B09359048091EB039091EC030F970A
:1046000034F488E19CEF9093B8078093B7078091CA
:10461000EB039091EC03079734F480E398EF9093C9
:10462000B8078093B7071A30A9F48091EB039091F3
:10463000EC03835F934034F088EE93E09093B807E7
:104640008093B7078091EB039091EC038A5F9340CE
:10465000DCF014C08091EB039091EC03855E9740F1
:1046600034F088EE93E09093B8078093B707809179
:10467000EB039091EC03835F974034F080ED97E07B
:104680009093B8078093B7078FEE80937A0080915C
:104690004A0490914B04A0914C04B0914D04809336
:1046A0005E0490935F04A0936004B09361048091D2
:1046B0005A0490915B04A0915C04B0915D048093D6
:1046C0007A0490937B04A0937C04B0937D04809142
:1046D000520490915304A0915404B09155048093D6
:1046E000720490937304A0937404B0937504809142
:1046F000560490915704A0915804B09159048093A6
:10470000760490937704A0937804B0937904809111
:104710004E0490914F04A0915004B09151048093A5
:104720006E0490936F04A0937004B0937104809111
:104730006D0787FF6EC0992009F06BC080911B0444
:10474000882309F066C08091B7079091B807893C2B
:1047500091058CF02091B7073091B807220F331FD5
:10476000220F331F8091B7079091B807820F931FD4
:104770008052934017C08091B7079091B807885333
:104780009F4FA4F42091B7073091B807220F331F31
:10479000220F331F8091B7079091B807820F931FA4
:1047A000805E9C4F9093B8078093B7078091AD07C8
:1047B0009091AE07893C91058CF02091AD07309126
:1047C000AE07220F331F220F331F8091AD07909148
:1047D000AE07820F931F8052934017C08091AD07A0
:1047E0009091AE0788539F4FA4F42091AD0730916C
:1047F000AE07220F331F220F331F8091AD07909118
:10480000AE07820F931F805E9C4F9093AE078093FC
:10481000AD0780916907E82FFF27EE0FFF1FE75CC8
:10482000F84F8081918182599F4F209135043091BA
:104830003604281739071CF42F5F3F4F0CC08081C6
:10484000918182599F4F821793074CF421153105AE
:1048500031F021503040309336042093350480915C
:104860006A07E82FFF27EE0FFF1FE75CF84F8081F4
:10487000918182599F4F209133043091340428173D
:1048800039071CF42F5F3F4F0CC080819181825902
:104890009F4F821793074CF42115310531F02150B9
:1048A0003040309334042093330480916B07E82F19
:1048B000FF27EE0FFF1FE75CF84F8081918182593F
:1048C0009F4F2091310430913204281739071CF48E
:1048D0002F5F3F4F0CC08081918182599F4F82177B
:1048E00093074CF42115310531F0215030403093BD
:1048F00032042093310480916C07E82FFF27EE0FDC
:10490000FF1FE75CF84F8081918182599F4F209172
:104910002F0430913004281739071CF42F5F3F4FC4
:104920000CC08081918182599F4F821793074CF46C
:104930002115310531F0215030403093300420935F
:104940002F04809135049091360497FF05C0109292
:104950003604109235040AC08F3F910539F034F0C7
:104960008FEF90E090933604809335048091330468
:104970009091340497FF05C01092340410923304D0
:104980000AC08F3F910539F034F08FEF90E090939B
:10499000340480933304809131049091320497FF62
:1049A00005C010923204109231040AC08F3F910565
:1049B00039F034F08FEF90E090933204809331041B
:1049C00080912F049091300497FF05C0109230041D
:1049D00010922F040AC08F3F910539F034F08FEF09
:1049E00090E09093300480932F04DF91CF911F913A
:1049F0000F91FF90EF90DF90CF90BF90AF909F907E
:104A0000089580912504882301F58093B60780934B
:104A1000AF078093D0078093D2078091B203882399
:104A200011F08093AF078091B303882311F0809336
:104A3000B6078091B403882311F08093D207809148
:104A4000B503882311F08093D0078091AF07992791
:104A50009093F6068093F5068091B6079927909378
:104A6000F8068093F7068091D20799279093FA066B
:104A70008093F9068091D00799279093FC06809344
:104A8000FB061092FC031092FB030E94A5170895E9
:104A90001F93809170078B3F98F08B3F19F48091A2
:104AA00035040EC08C3F19F48091330409C08D3F4A
:104AB00019F48091310404C08E3F21F480912F04B9
:104AC00080937E0380917E03882321F08F3F11F431
:104AD00080937E0380916F078B3F98F08B3F19F492
:104AE000809135040EC08C3F19F48091330409C0C5
:104AF0008D3F19F48091310404C08E3F21F48091E0
:104B00002F0480937F0380917F03882329F08436CC
:104B100018F084E680937F03809171078B3F98F0B3
:104B20008B3F19F4809135040EC08C3F19F48091AD
:104B3000330409C08D3F19F48091310404C08E3FC5
:104B400021F480912F0480937D0380917D0388233D
:104B500029F0843618F084E680937D0380917307F2
:104B60008B3F98F08B3F19F4809135040EC08C3F39
:104B700019F48091330409C08D3F19F480913104F8
:104B800004C08E3F21F480912F0480937C03809198
:104B90007C03882321F08F3F11F480937C03809164
:104BA0007A078B3F98F08B3F19F4809135040EC043
:104BB0008C3F19F48091330409C08D3F19F4809122
:104BC000310404C08E3F21F480912F0480937B0335
:104BD00080917B03882321F08F3F11F480937B0326
:104BE00080917B078B3F98F08B3F19F480913504BF
:104BF0000EC08C3F19F48091330409C08D3F19F425
:104C00008091310404C08E3F21F480912F04809361
:104C10007A0380917A038B3010F48AE002C08F3FD0
:104C200011F480937A0380917C078B3F98F08B3F3F
:104C300019F4809135040EC08C3F19F4809133042F
:104C400009C08D3F19F48091310404C08E3F21F4D6
:104C500080912F048093790380917903882321F038
:104C60008F3F11F480937903809181078B3F98F0F7
:104C70008B3F19F4809135040EC08C3F19F480915C
:104C8000330409C08D3F19F48091310404C08E3F74
:104C900021F480912F0480937703809177038823F8
:104CA00021F08F3F11F480937703809182078B3F2F
:104CB00098F08B3F19F4809135040EC08C3F19F4A5
:104CC0008091330409C08D3F19F48091310404C0F0
:104CD0008E3F21F480912F04809316048091160456
:104CE000882321F08F3F11F480931604809183076D
:104CF0008B3F98F08B3F19F4809135040EC08C3FA8
:104D000019F48091330409C08D3F19F48091310466
:104D100004C08E3F21F480912F048093150480916C
:104D20001504882321F08F3F11F48093150480919E
:104D300084078B3F98F08B3F19F4809135040EC0A7
:104D40008C3F19F48091330409C08D3F19F4809190
:104D5000310404C08E3F21F480912F048093140409
:104D600080911404882321F08F3F11F48093140460
:104D7000809185078B3F98F08B3F19F48091350423
:104D80000EC08C3F19F48091330409C08D3F19F493
:104D90008091310404C08E3F21F480912F048093D0
:104DA000130480911304882321F08F3F11F4809322
:104DB0001304809195078B3F98F08B3F19F48091F5
:104DC00035040EC08C3F19F48091330409C08D3F27
:104DD00019F48091310404C08E3F21F480912F0496
:104DE0008093120480911204882321F08F3F11F4E4
:104DF00080931204809196078B3F98F08B3F19F4B3
:104E0000809135040EC08C3F19F48091330409C0A1
:104E10008D3F19F48091310404C08E3F21F48091BC
:104E20002F048093110480911104882321F08F3F77
:104E300011F480931104809197078B3F98F08B3F7A
:104E400019F4809135040EC08C3F19F4809133041D
:104E500009C08D3F19F48091310404C08E3F21F4C4
:104E600080912F048093100480911004882321F0F6
:104E70008F3F11F480931004809198078B3F98F036
:104E80008B3F19F4809135040EC08C3F19F480914A
:104E9000330409C08D3F19F48091310404C08E3F62
:104EA00021F480912F0480930F0480910F048823B4
:104EB00021F08F3F11F480930F04809186078B3F80
:104EC00098F08B3F19F4809135040EC08C3F19F493
:104ED0008091330409C08D3F19F48091310404C0DE
:104EE0008E3F21F480912F04809376038091760386
:104EF000882321F08F3F11F48093760380918B07F4
:104F00008B3F98F08B3F19F4809135040EC08C3F95
:104F100019F48091330409C08D3F19F48091310454
:104F200004C08E3F21F480912F04809375038091FB
:104F30007503882321F08F3F11F4809375038091CE
:104F40008E078B3F98F08B3F19F4809135040EC08B
:104F50008C3F19F48091330409C08D3F19F480917E
:104F6000310404C08E3F21F480912F0480930E04FD
:104F700080910E04882321F08F3F11F480930E045A
:104F800080918F078B3F98F08B3F19F48091350407
:104F90000EC08C3F19F48091330409C08D3F19F481
:104FA0008091310404C08E3F21F480912F048093BE
:104FB0000D0480910D04882321F08F3F11F480931C
:104FC0000D04809194078B3F98F08B3F19F48091EA
:104FD00035040EC08C3F19F48091330409C08D3F15
:104FE00019F48091310404C08E3F21F480912F0484
:104FF0008093740380917403882321F08F3F11F410
:105000008093740310917703812F992787FD9095E2
:10501000A92FB92FBC01CD010E94EE4217FF06C097
:1050200020E030E040E853E40E94494227E137EBBA
:1050300041ED58E30E946843DC01CB01809380037B
:1050400090938103A0938203B093830380917807A8
:105050008093D707809177078093B9071F910895B0
:105060002F923F924F925F926F927F928F929F9278
:10507000AF92BF92CF92DF92EF92FF920F931F9366
:10508000CF93DF93CDB7DEB765970FB6F894DEBF49
:105090000FBECDBF0E945B1E299AE0902604F090BF
:1050A0002704FA82E9828091B90799270A96E816BF
:1050B000F90614F49A83898380912E04843608F0CB
:1050C0006EC080910303882399F480910603909128
:1050D00007038F5F9F4F61F488E99AE39093CE03B3
:1050E0008093CD0380E09CE09093070380930603B8
:1050F0008091B8049091B904009731F00197909392
:10510000B9048093B80404C01092250410923B04A3
:10511000809101018A3011F4289A01C02898809169
:10512000010490910204895E9340B0F180917E0762
:10513000282F33273A83298381E080933B04809191
:105140006507A82FBB27AA0FBB1FFD01E15BF84F26
:105150001182108280916607282F3327220F331F78
:10516000C901815B984FFC0111821082A75CB84F86
:1051700011961C921E92275C384FD90111961C92F1
:105180001E9280916807E82FFF27EE0FFF1FE75C54
:10519000F84F11821082A3C210922504A0C2809100
:1051A0002E048D3808F49BC210923B0490917F0727
:1051B00082E3989FC00111249093B9048093B804AE
:1051C000E981FA81B9976CF0809101049091020411
:1051D000FFEF8F3F9F0729F0019690930204809381
:1051E000010480910104909102048F3F910509F020
:1051F00070F510929C0410929D0410929E041092DF
:105200009F041092A0041092A1041092A204109284
:10521000A3048A3F9105D9F481E08093C0041092E1
:10522000A4041092A5041092A6041092A704109250
:105230004A0410924B0410924C0410924D041092A8
:105240004604109247041092480410924904809139
:105250006707E82FFF27EE0FFF1FE75CF84F8081FD
:105260009181813591050CF491C12091250422236F
:1052700009F08CC180916807E82FFF27EE0FFF1F10
:10528000E75CF84F808191818C3491050CF4F5C076
:105290008091BA048F5F8093BA04893C08F476C188
:1052A00029982093BA0410920204109201043091BC
:1052B0006507E32FFF27EE0FFF1FE75CF84F8081A4
:1052C000918187349105B4F480916607E82FFF2718
:1052D000EE0FFF1FE75CF84F808191810190F08114
:1052E000E02DF7FF03C0F095E195FF4FE734F1059E
:1052F0000CF47AC041E020916607A22FBB27AA0FC9
:10530000BB1FA75CB84F8D919C9111978734910575
:1053100044F0E32FFF27EE0FFF1FE75CF84F80817B
:1053200091818D919C918734910574F080916507EE
:10533000E82FFF27EE0FFF1FE75CF84F8081918178
:10534000873491050CF042E0E22FFF27EE0FFF1F9C
:10535000E75CF84F808191818634910574F48091E7
:105360006507E82FFF27EE0FFF1FE75CF84F8081EE
:105370009181873491050CF043E0E22FFF27EE0F77
:10538000FF1FE75CF84F808191818A5B9F4F74F427
:1053900080916507E82FFF27EE0FFF1FE75CF84FAE
:1053A00080819181873491050CF044E0E22FFF2742
:1053B000EE0FFF1FE75CF84F808191818A5B9F4F62
:1053C00074F480916507E82FFF27EE0FFF1FE75C5D
:1053D000F84F80819181863491050CF445E0A2E07C
:1053E000B0E0042E0E94474480916607E82FFF2713
:1053F000EE0FFF1FE75CF84F808191810190F081F3
:10540000E02DF7FF03C0F095E195FF4F7497BCF4D2
:1054100080916507E82FFF27EE0FFF1FE75CF84F2D
:10542000808191818A5B9F4F54F481E0809336069E
:1054300088EE93E09093CE038093CD03A7C00E94A3
:10544000790247E465E677E00E944F0280916D079C
:1054500080FF10C080910E0390910F03875B9340F3
:1054600038F480910E0390910F038E5E924010F4F9
:105470000E94D80E0E94C21C82C080819181855BEF
:105480009F4F0CF081C08091BA048F5F8093BA0463
:10549000893C08F47BC02998A4E0B0E08FEF082E87
:1054A0000E944744209325042093BA0410920204DA
:1054B000109201040E94C21CA4E0B0E08091880414
:1054C0009091890497FF02C081509F4F892F990FB7
:1054D000990B082E0E944744A5E0B0E08091880413
:1054E00090918904082E0E944744A6E0B0E0809184
:1054F00086049091870497FF02C081509F4F892FA7
:10550000990F990B082E0E944744A7E0B0E08091C4
:10551000860490918704082E0E94474408E010E01A
:105520008091800490918104A0918204B0918304C1
:10553000BC01CD010E94D142DC01CB019C0197FF4F
:1055400002C021503F4F832F992787FD9A95D8019C
:10555000082E0E94474409E010E080918004909159
:105560008104A0918204B0918304BC01CD010E940A
:10557000D142DC01CB01D801082E0E9447440E9491
:1055800079020E94471B02C02093BA0480916707EA
:10559000E82FFF27EE0FFF1FE75CF84F8081918116
:1055A0008B5A9F4F0CF09BC020916807E22FFF277A
:1055B000EE0FFF1FE75CF84F80819181855B9F4F65
:1055C0000CF06DC08091BB048F5F8093BB04893C5D
:1055D00008F467C088EC8093BB0481E090E090936E
:1055E00002048093010481E0809325041092A404B6
:1055F0001092A5041092A6041092A70410924A04D7
:1056000010924B0410924C0410924D0410924604D8
:1056100010924704109248041092490410925A04C0
:1056200010925B0410925C0410925D04109252047C
:1056300010925304109254041092550480917A04ED
:1056400090917B04A0917C04B0917D0480935604DA
:1056500090935704A0935804B09359048091720416
:1056600090917304A0917404B091750480934E04DA
:1056700090934F04A0935004B093510410929C0453
:1056800010929D0410929E0410929F041092A00408
:105690001092A1041092A2041092A30402C01092CE
:1056A000BB04E22FFF27EE0FFF1FE75CF84F80815E
:1056B00091818C3491058CF08091BC048F5F809334
:1056C000BC04893C60F01092250488EC8093BC04F3
:1056D000109202041092010402C01092BC04809146
:1056E0007103815080937103809171038F3F29F082
:1056F00080913B04882309F4DFC30E9448258091F0
:10570000C9049091CA04AC01440F551F480F591F9A
:10571000F0906507AF2DBB27AA0FBB1FFD01E75C0B
:10572000F84FE0907407CE2CDD24808191818C9D10
:1057300080018D9D100D9C9D100D1124400F511F57
:1057400057FF02C04D5F5F4F55954795559547955B
:10575000A15BB84F80917507682F77278D919C9139
:10576000869F9001879F300D969F300D1124420F28
:10577000531F5093CA044093C9048091F10490913F
:10578000F2042091ED043091EE04820F931F481B28
:10579000590B50932D0440932C048091CB0490918D
:1057A000CC04AC01440F551F480F591F00916607E8
:1057B000A02FBB27AA0FBB1FFD01E75CF84F80811C
:1057C00091818C9DF0018D9DF00D9C9DF00D11241B
:1057D0004E0F5F1F57FF02C04D5F5F4F55954795B6
:1057E00055954795A15BB84F8D919C91869F9001EF
:1057F000879F300D969F300D1124420F531F5093F9
:10580000CC044093CB048091EF049091F00420915C
:10581000EB043091EC04820F931F481B590B5093FB
:105820002B0440932A0480916807E82FFF27EE0F8E
:10583000FF1FE75CF84F80819181909581959F4F84
:10584000909329048093280480916707E82FFF270D
:10585000EE0FFF1FE75CF84F8081918188589F4FC2
:10586000909327048093260410917A03812F99271F
:1058700087FD9095A92FB92FBC01CD010E94EE4262
:1058800017FF06C020E030E040E853E40E944942A0
:1058900020E030E040E251E40E944942DC01CB01CB
:1058A00020E030E040E85CE3BC01CD010E946843A9
:1058B000DC01CB018093DC079093DD07A093DE072A
:1058C000B093DF0710917903812F992787FD909579
:1058D000A92FB92FBC01CD010E94EE4217FF06C0CF
:1058E00020E030E040E853E40E94494220E030EEFE
:1058F0004BE256E40E948B42DC01CB018093CC0743
:105900009093CD07A093CE07B093CF076091AF03DC
:10591000662331F08AE090E09093CE038093CD032C
:10592000462F552742FF09C080910F04282F3327A7
:10593000220F331F220F331F13C09A0128703070BB
:1059400043FF0EC080910F04282F33278CEF9FEF69
:10595000289FA001299F500D389F500D11249A01B6
:1059600080910B0490910C04AC01F3E0440F551F9F
:10597000FA95E1F7481B590B420F531F57FF02C01E
:10598000495F5F4FE3E055954795EA95E1F75093FE
:105990000C0440930B04462F552744FF09C0809107
:1059A0000F04282F3327220F331F220F331F13C05A
:1059B0009A012072307045FF0EC080910F04282F8D
:1059C00033278CEF9FEF289FD001299FB00D389F80
:1059D000B00D11249D018091090490910A04AC013D
:1059E00063E0440F551F6A95E1F7481B590B420FBE
:1059F000531F57FF02C0495F5F4F83E0559547959E
:105A00008A95E1F750930A04409309044091AE034C
:105A1000842F992783FF03C082E390E007C09C0195
:105A20002470307082FF07C08EEC9FEF90930804C3
:105A30008093070404C03093080420930704242FA4
:105A4000332721FF09C0809172039091730301965F
:105A5000909373038093720324FF09C080917203B3
:105A600090917303019790937303809372038091D5
:105A70000B0490910C0497FD019695958795E09104
:105A80002C04F0912D04E80FF91FF0932D04E093FE
:105A90002C048091090490910A0497FD0196959534
:105AA000879560912A0470912B04680F791F709379
:105AB0002B0460932A048091070490910804880FB6
:105AC000991F880F991F4091280450912904480F6D
:105AD000591F50932904409328048091420680FF67
:105AE00059C080910F04813808F454C080913B065E
:105AF000992787FD90952E2D3327829FD001839F74
:105B0000B00D929FB00D1124EA0FFB1FF0932D04EE
:105B1000E0932C0480913C06992787FD9095829F05
:105B2000F001839FF00D929FF00D11246E0F7F1FE7
:105B300070932B0460932A0480913D06992787FD7A
:105B40009095480F591F5093290440932804809141
:105B50003F06282F332727FD30958091720799271C
:105B6000289FA001299F500D389F500D112450935C
:105B700073034093720380913E06282F3327809150
:105B80002604909127042817390724F4309327041A
:105B900020932604809126049091270497FF04C047
:105BA000109227041092260480916D0782FF0CC08A
:105BB00080E090E0A0E0B0E08093CC079093CD0728
:105BC000A093CE07B093CF078091DC079091DD07BB
:105BD000A091DE07B091DF0720E030E040E050E028
:105BE000BC01CD010E94F842882364F480E090E07B
:105BF000A0E0B0E08093DC079093DD07A093DE0780
:105C0000B093DF078091CC079091CD07A091CE078C
:105C1000B091CF0720E030E040E050E0BC01CD0182
:105C20000E94F842882364F480E090E0A0E0B0E0B5
:105C30008093CC079093CD07A093CE07B093CF0766
:105C400040912C0450912D04CA0157FD03969C01EC
:105C5000359527953595279537FF03C030952195C4
:105C60003F4F8091050490910604821793076CF4CE
:105C7000CA0157FF03C0909581959F4F97FD0396EA
:105C8000959587959595879501C001979093060402
:105C90008093050440912A0450912B04CA0157FDBA
:105CA00003969C01359527953595279537FF03C0B9
:105CB000309521953F4F8091030490910404821701
:105CC00093076CF4CA0157FF03C0909581959F4FCD
:105CD00097FD0396959587959595879501C00197B2
:105CE000909304048093030480913B04882341F043
:105CF00010920604109205041092040410920304FA
:105D0000E02FFF27EE0FFF1FE75CF84F40918C0755
:105D1000242F3327808191812817390744F48091FB
:105D2000990782FF04C081E080931A0413C0E02F1A
:105D3000FF27EE0FFF1FE75CF84F842F9927209174
:105D40008D07821B9109208131812817390714F4AE
:105D500010921A0440916607E42FFF27EE0FFF1FF1
:105D6000E75CF84F50918C07852F9927222733271E
:105D7000281B390B808191818217930744F480910D
:105D8000990783FF04C081E08093190416C08091B5
:105D90001904882391F0E42FFF27EE0FFF1FE75C23
:105DA000F84F80918D079927851B910920813181BA
:105DB0008217930714F410921904EF2DFF27EE0FAA
:105DC000FF1FE75CF84F40918C07242F3327808119
:105DD00091812817390744F48091990780FF04C006
:105DE00081E08093170417C080911704882399F0ED
:105DF000EF2DFF27EE0FFF1FE75CF84F842F992749
:105E000020918D07821B9109208131812817390744
:105E100014F41092170440916507E42FFF27EE0F4A
:105E2000FF1FE75CF84F50918C07852F9927222799
:105E30003327281B390B808191818217930744F403
:105E40008091990781FF04C081E08093180416C0F7
:105E500080911804882391F0E42FFF27EE0FFF1F95
:105E6000E75CF84F80918D079927851B9109208168
:105E700031818217930714F41092180480911A0448
:105E8000882319F480911904811181E080931B0407
:105E900080911704882321F480911804882351F0FD
:105EA00081E080931C0410921B0410921A0410923B
:105EB000190402C080931C0420911B04222331F09A
:105EC00084E690E09093CE038093CD03222321F4C7
:105ED00080911C04882351F080918B079927A98118
:105EE000BA818A179B0714F49A838983B0913B0483
:105EF000BB83BB2341F11092290410922804109215
:105F00002D0410922C0410922B0410922A0480E08D
:105F100090E0A8ECBFE38093DC079093DD07A093AB
:105F2000DE07B093DF078BE09CEBA2E3BCE380933A
:105F3000CC079093CD07A093CE07B093CF071092D4
:105F40001B0410921C048091C2079091C307A0917A
:105F5000C407B091C50720917A0430917B04409129
:105F60007C0450917D04820F931FA41FB51F809362
:105F7000C2079093C307A093C407B093C50780914D
:105F8000C8079091C907A091CA07B091CB0760904C
:105F90007204709073048090740490907504860D60
:105FA000971DA81DB91D8093C8079093C907A0939A
:105FB000CA07B093CB078091BA079091BB07A09115
:105FC000BC07B091BD07E0907604F0907704009193
:105FD000780410917904EC82FD820E831F838E0D6C
:105FE0009F1DA01FB11F8093BA079093BB07A0937A
:105FF000BC07B093BD078091B2079091B307A09101
:10600000B407B091B507E0906E04F0906F04009172
:10601000700410917104E886F9860A871B878E0D3B
:106020009F1DA01FB11F8093B2079093B307A09349
:10603000B407B093B50750901C04552029F4809103
:106040001B04882309F45FC010926A0410926B0449
:1060500010926C0410926D04109266041092670402
:1060600010926804109269041092C2071092C3073C
:106070001092C4071092C5071092C8071092C90762
:106080001092CA071092CB071092BA071092BB0762
:106090001092BC071092BD071092B2071092B3077E
:1060A0001092B4071092B50780915A0490915B0446
:1060B000A0915C04B0915D048093560490935704C2
:1060C000A0935804B09359048091520490915304C2
:1060D000A0915404B091550480934E0490934F04C2
:1060E000A0935004B09351041092D8031092D70398
:1060F00010921E0410921D041092200410921F048E
:10610000552009F0FBC080911B04882309F0F6C0DC
:1061100080917907E82EFF2400271127CA01B901D1
:10612000A80197010E94244459016A018091D50772
:106130009091D607AA2797FDA095BA2FA81AB90A59
:10614000CA0ADB0AC401B301A80197010E942444D2
:1061500079018A018091E5079091E607AA2797FDCA
:10616000A095BA2FE81AF90A0A0B1B0BD601C50134
:10617000D7FE03C00F96A11DB11D5C016D0154E057
:10618000D594C794B794A7945A95D1F7D801C7016D
:1061900017FF03C00F96A11DB11D7C018D0144E0C6
:1061A00015950795F794E7944A95D1F780910504E2
:1061B00090910604819734F4809103049091040433
:1061C0008197A4F0C601B50123E030E040E050E043
:1061D0000E94244459016A01C801B70123E030E05C
:1061E00040E050E00E94244479018A0180916807D0
:1061F000E82FFF27EE0FFF1FE75CF84F80819181AA
:106200000190F081E02DF7FF03C0F095E195FF4F7D
:106210007A97A4F0C601B50123E030E040E050E0F9
:106220000E94244459016A01C801B70123E030E00B
:1062300040E050E00E94244479018A0121E2A21644
:10624000B104C104D1042CF030E2A32EB12CC12C36
:10625000D12C30EEA3163FEFB3063FEFC3063FEF5E
:10626000D30644F420EEA22E2FEFB22E2FEFC22E33
:106270002FEFD22E41E2E416F104010511052CF0B6
:1062800090E2E92EF12C012D112D50EEE5165FEF75
:10629000F5065FEF05075FEF150744F480EEE82E83
:1062A0008FEFF82E8FEF082F8FEF182F80915A0461
:1062B00090915B04A0915C04B0915D048A199B09E4
:1062C000AC09BD0980935A0490935B04A0935C04CD
:1062D000B0935D048091520490915304A0915404B2
:1062E000B09155048E199F09A00BB10B80935204F5
:1062F00090935304A0935404B09355048091D70312
:106300009091D8038F3F910509F008F474C555208A
:1063100009F0F1C480911B04882309F0ECC480913A
:106320003904882309F0E7C48091C2079091C3071C
:10633000A091C407B091C507B7FF04C081509F4F1B
:10634000AF4FBF4F292E3A2E4B2E552447FC5A945F
:106350002092C2073092C3074092C4075092C507EB
:106360008091C8079091C907A091CA07B091CB0747
:10637000B7FF04C081509F4FAF4FBF4F892F9A2F57
:10638000AB2FBB27A7FDBA958C879D87AE87BF87AC
:106390008093C8079093C907A093CA07B093CB070F
:1063A00080917907E82EFF240027112720916A04A5
:1063B00030916B0440916C0450916D04C801B70199
:1063C0000E94B04397FF04C061507F4F8F4F9F4F93
:1063D000A72EB82EC92EDD24C7FCDA94A0926A0439
:1063E000B0926B04C0926C04D0926D04209166044C
:1063F000309167044091680450916904C801B70165
:106400000E94B04397FF04C061507F4F8F4F9F4F52
:10641000672E782E892E992487FC9A9460926604C0
:10642000709267048092680490926904809162047B
:1064300090916304A0916404B0916504B7FF04C017
:1064400081509F4FAF4FBF4F892F9A2FAB2FBB2744
:10645000A7FDBA958093620490936304A0936404AB
:10646000B0936504D201C1018A199B09AC09BD0929
:106470008093B0049093B104A093B204B093B3049A
:1064800020919207E22EFF2400271127BC01CD01A5
:10649000A80197010E94244459016A012093C10474
:1064A0003093C2044093C3045093C4048C859D85EB
:1064B000AE85BF8586199709A809B9098093B404E8
:1064C0009093B504A093B604B093B704BC01CD017A
:1064D000A80197010E9424442093C5043093C60468
:1064E0004093C7045093C804D601C501D7FE04C029
:1064F00081509F4FAF4FBF4F892F9A2FAB2FBB2794
:10650000A7FDBA9590931E0480931D0457FF04C005
:1065100021503F4F4F4F5F4FBB2757FDBA95A52FD7
:10652000942F832F9093200480931F04809105045F
:10653000909106048197D4F480910304909104040F
:106540008197A4F480916807E82FFF27EE0FFF1FC3
:10655000E75CF84F808191810190F081E02DF7FF99
:1065600003C0F095E195FF4F7A97C4F080911D0428
:1065700090911E0497FD01969595879590931E0422
:1065800080931D0480911F049091200497FD019633
:10659000959587959093200480931F048091BA0766
:1065A0009091BB07A091BC07B091BD07B7FF04C095
:1065B00081509F4FAF4FBF4F892F9A2FAB2FBB27D3
:1065C000A7FDBA958093BA079093BB07A093BC0729
:1065D000B093BD078091B2079091B307A091B40723
:1065E000B091B507B7FF04C081509F4FAF4FBF4F69
:1065F000892F9A2FAB2FBB27A7FDBA958093B2079F
:106600009093B307A093B407B093B50780917A0431
:1066100090917B04A0917C04B0917D04EC80FD807E
:106620000E811F81E81AF90A0A0B1B0BE092A804DD
:10663000F092A9040093AA041093AB048091720411
:1066400090917304A0917404B091750428853985E4
:106650004A855B85281B390B4A0B5B0B2093AC04E6
:106660003093AD044093AE045093AF04E092B00475
:10667000F092B1040093B2041093B3042093B404D5
:106680003093B5044093B6045093B70480915604F8
:1066900090915704A0915804B09159048E199F0904
:1066A000A00BB10B8093560490935704A093580409
:1066B000B093590480914E0490914F04A0915004DE
:1066C000B0915104821B930BA40BB50B80934E0425
:1066D00090934F04A0935004B09351042091370439
:1066E00030913804213831054CF080918E0490911E
:1066F0008F04019690938F0480938E0420583F4F0F
:106700004CF480918E0490918F04019790938F04A4
:1067100080938E04A090C807B090C907C090CA07A4
:10672000D090CB07C601B5012AE130E040E050E04F
:106730000E94244430930A072093090710923804DA
:106740001092370481E090E09093CE048093CD04C2
:106750008091D3049091D404A091D504B091D60433
:106760002091C2073091C3074091C4075091C507DB
:10677000821B930BA40BB50B815E914BAF4FBF4FA8
:106780008F539C49A040B04008F0FEC0F1E0EF16E6
:10679000F0E1FF06F0E00F07F0E01F070CF46CC01B
:1067A0008091CF04882309F463C0D801C70117FF83
:1067B00007C088279927DC018E199F09A00BB10B10
:1067C000B7FF04C08150904FAF4FBF4F2CE0B5953D
:1067D000A795979587952A95D1F701969093CE0422
:1067E0008093CD04D801C70117FF03C00796A11DF0
:1067F000B11D13E0B595A795979587951A95D1F793
:106800008093C1049093C204A093C304B093C404C2
:1068100089589341A040B04064F088E893E1A0E03B
:10682000B0E08093C1049093C204A093C304B093DA
:10683000C4042091C1043091C2044091C30450911A
:10684000C40457FF04C021503F4F4F4F5F4F232FC9
:10685000342F452F552747FD5A9580911D0490915F
:106860001E04820F931F90931E0480931D0406C084
:1068700081E08093CF0402C01092CF04E090B00476
:10688000F090B1040091B2041091B30420E0E2163C
:1068900020EFF2062FEF02072FEF12070CF071C066
:1068A0008091D004882309F468C0A801970117FFDC
:1068B00007C022273327A9012E193F09400B510B8E
:1068C00057FF04C02150304F4F4F5F4FECE05595BC
:1068D000479537952795EA95D1F78091CD0490910A
:1068E000CE04820F931F9093CE048093CD04D801E1
:1068F000C70117FF03C00796A11DB11D73E0B59531
:10690000A795979587957A95D1F78093C104909331
:10691000C204A093C304B093C40488579C4EAF4FE5
:10692000BF4F64F488E79CEEAFEFBFEF8093C104E4
:106930009093C204A093C304B093C4042091C104F3
:106940003091C2044091C3045091C40457FF04C065
:1069500021503F4F4F4F5F4F232F342F452F552747
:1069600047FD5A9580911D0490911E04820F931F3C
:1069700090931E0480931D0411C081E08093D00485
:106980000DC01092D0040AC01092CE041092CD0413
:1069900084EF91E090938D0380938C031091930783
:1069A000212F33278091CD049091CE0428173907E9
:1069B00024F43093CE042093CD044091B004509140
:1069C000B1046091B2047091B304413084E058077F
:1069D00080E0680780E0780774F0809192049091DD
:1069E00093042091CD043091CE04820F931F909395
:1069F00093048093920440505C4F6F4F7F4F74F428
:106A000080919204909193042091CD043091CE0412
:106A1000821B930B909393048093920481E090E007
:106A20009093CE048093CD041092C5041092C604B6
:106A30001092C7041092C8048091D7049091D80492
:106A4000A091D904B091DA048A199B09AC09BD0957
:106A5000815E914BAF4FBF4F8F539C49A040B040D8
:106A600008F000C1C090B404D090B504E090B60422
:106A7000F090B704F1E0CF16F0E1DF06F0E0EF06AA
:106A8000F0E0FF060CF46CC08091D104882309F477
:106A900063C0D701C601F7FE07C088279927DC012C
:106AA0008C199D09AE09BF09B7FF04C08150904FF2
:106AB000AF4FBF4F2CE0B595A795979587952A9531
:106AC000D1F701969093CE048093CD04D701C601EF
:106AD000F7FE03C00796A11DB11D03E0B595A7956C
:106AE000979587950A95D1F78093C5049093C6042E
:106AF000A093C704B093C80489589341A040B04004
:106B000064F088E893E1A0E0B0E08093C50490933E
:106B1000C604A093C704B093C8042091C504309163
:106B2000C6044091C7045091C80457FF04C02150C7
:106B30003F4F4F4F5F4F232F342F452F552747FD92
:106B40005A9580911F0490912004820F931F909377
:106B5000200480931F0406C081E08093D10402C00A
:106B60001092D10420E0C21620EFD2062FEFE206E9
:106B70002FEFF2060CF073C08091D204882309F441
:106B80006AC0D701C601F7FE07C088279927DC0134
:106B90008C199D09AE09BF099C01AD01B7FF04C066
:106BA0002150304F4F4F5F4FECE05595479537954B
:106BB0002795EA95D1F78091CD049091CE04820F6C
:106BC000931F9093CE048093CD04D701C601F7FEA6
:106BD00003C00796A11DB11D73E0B595A7959795C4
:106BE00087957A95D1F78093C5049093C604A093B6
:106BF000C704B093C80488579C4EAF4FBF4F64F48E
:106C000088E79CEEAFEFBFEF8093C5049093C60476
:106C1000A093C704B093C8042091C5043091C60462
:106C20004091C7045091C80457FF04C021503F4F02
:106C30004F4F5F4F232F342F452F552747FD5A9530
:106C400080911F0490912004820F931F9093200441
:106C500080931F0411C081E08093D2040DC0109274
:106C6000D2040AC01092CE041092CD0484EF91E0B9
:106C700090938D0380938C03212F33278091CD0433
:106C80009091CE042817390724F43093CE04209332
:106C9000CD044091B4045091B5046091B604709154
:106CA000B704413084E0580780E0680780E0780747
:106CB00074F080919004909191042091CD043091D2
:106CC000CE04820F931F90939104809390044050C0
:106CD0005C4F6F4F7F4FCCF4809190049091910462
:106CE0002091CD043091CE04821B930B909391049C
:106CF000809390040AC01092200410921F041092F6
:106D00001E0410921D04109239048091CC079091BA
:106D1000CD07A091CE07B091CF0720E030E040E052
:106D200050E0BC01CD010E94F842882341F410924A
:106D3000200410921F0410921E0410921D048091D2
:106D4000C2079091C307A091C407B091C507809373
:106D5000D3049093D404A093D504B093D604809127
:106D6000C8079091C907A091CA07B091CB0780933B
:106D7000D7049093D804A093D904B093DA04109266
:106D80006A0410926B0410926C0410926D041092BD
:106D900066041092670410926804109269041092BD
:106DA00062041092630410926404109265041092BD
:106DB000C2071092C3071092C4071092C507109221
:106DC000C8071092C9071092CA071092CB071092F9
:106DD000BA071092BB071092BC071092BD07109221
:106DE000B2071092B3071092B4071092B507109231
:106DF000D8031092D703A0902804B0902904C501AD
:106E0000B7FE04C0882799278A199B094097ACF0E0
:106E100080916D0784FD11C081E08093C004809152
:106E2000E1079091E20790933F0480933E048AEF3C
:106E300090E090938D0380938C03D0907607ED2C97
:106E4000FF2400271127B501882777FD8095982F0B
:106E50009501B7FE04C0222733272A193B0944278E
:106E600037FD4095542F0E94B0439B01AC01C801EF
:106E7000B7010E94B04397FF04C061507E4F8F4F0F
:106E80009F4F59E095958795779567955A95D1F7D6
:106E90009B018D2D99278A9DD0018B9DB00D9A9DC8
:106EA000B00D1124CD01B7FD039695958795959565
:106EB0008795280F391F442737FD4095542F20937D
:106EC000A4043093A5044093A6045093A704809192
:106ED0004A0490914B04A0914C04B0914D04821B44
:106EE000930BA40BB50B80934A0490934B04A0938F
:106EF0004C04B0934D048155934CA040B04064F0D5
:106F000080E593ECA0E0B0E080934A0490934B04BA
:106F1000A0934C04B0934D0480914A0490914B048B
:106F2000A0914C04B0914D04805B9C43AF4FBF4F88
:106F300064F480EB9CE3AFEFBFEF80934A0490933F
:106F40004B04A0934C04B0934D0480914004909165
:106F50004104892B09F465C180916D0783FF61C1EC
:106F600080917A0490917B04A0917C04B0917D047F
:106F7000B7FF04C081509E4FAF4FBF4F29E0B5957A
:106F8000A795979587952A95D1F74C0197FF04C04F
:106F900090948194910893948091720490917304D9
:106FA000A0917404B0917504B7FF04C081509E4F46
:106FB000AF4FBF4F09E0B595A795979587950A956F
:106FC000D1F7BC0197FF03C0709561957F4F86167E
:106FD00097060CF44B01B40197FE02C0695F7F4F26
:106FE0003B0113E0759467941A95E1F70894611CCE
:106FF000711C09E18016910434F58091C004882346
:1070000011F180918C0390918D03892BE1F488EC30
:1070100090E09093CE038093CD038091E10790910F
:10702000E207A091E307B091E407BC01CD012EE097
:1070300036E040E050E00E94244430933F04209327
:107040003E041092C0048091400490914104845EFB
:107050009D4F7C010027F7FC0095102FA090E107C1
:10706000B090E207C090E307D090E407C601B501F5
:107070002EE036E040E050E00E942444E21AF30A99
:10708000040B150BC801B70128E631E040E050E0E1
:107090000E942444DC01CB01FC01E45BF040CF0101
:1070A000B3E0880F991FBA95E1F7B3010E94EF434F
:1070B0009B01442737FD4095542F2A0D3B1D4C1D45
:1070C0005D1D2093E1073093E2074093E30750935F
:1070D000E40710917B03612F7727869EC001879E6E
:1070E000900D969E900D112497FDCF964C01A6E031
:1070F00095948794AA95E1F7681979094B011616BA
:1071000017060CF088C080918C0390918D03009736
:1071100009F07FC080913704909138048E0F9F1F33
:107120009093380480933704E0900504F0900604AF
:107130008091030490910404E80EF91EF7FE04C048
:1071400087E090E0E80EF91E63E0F594E7946A9515
:10715000E1F7A0E4B0E0EA0EFB1ECA01B9012EE09F
:1071600036E040E050E00E942444DA01C901209159
:107170003E0430913F04442737FD4095542F821B35
:10718000930BA40BB50B845E9D4FAF4FBF4FBC015B
:10719000CD0128E631E040E050E00E942444DC01CB
:1071A000CB01845B9040889DF001899DF00D989DF6
:1071B000F00D1124CF01B7010E94EF4383E0189F27
:1071C000400111248616970614F4B40108C08827DC
:1071D000992788199909681779070CF4BC019B0154
:1071E000442737FD4095542F80914A0490914B04D9
:1071F000A0914C04B0914D04820F931FA41FB51FA2
:1072000080934A0490934B04A0934C04B0934D0494
:1072100008C0019702C08AEF90E090938D0380939D
:107220008C038091BF0481508093BF048F3F09F08D
:10723000B0C088E18093BF0480917907E82EFF24D5
:107240000027112780917A0490917B04A0917C04FF
:10725000B0917D04BC01CD01A80197010E94244496
:107260003093DE062093DD068091720490917304C2
:10727000A0917404B0917504BC01CD01A8019701DF
:107280000E9424443093E0062093DF068091D507C6
:107290009091D6079093E2068093E1068091E507EE
:1072A0009091E6079093E4068093E3068091D807D7
:1072B0009091D9079093E6068093E5068091230488
:1072C000909124049093E8068093E706809142040D
:1072D00090914304A0914404B0914504B7FF04C0C9
:1072E00081509E4FAF4FBF4F39E0B595A795979509
:1072F00087953A95D1F79093EA068093E9068091B5
:107300004004909141049093EE068093ED068091A5
:107310001403909115039093F0068093EF068091EB
:10732000E1079091E207A091E307B091E407BC0167
:10733000CD012EE036E040E050E00E94244430933E
:10734000F4062093F30680912E0499279093F20679
:107350008093F1068091BE079091BF079093FE063F
:107360008093FD06809136069927909304078093B9
:1073700003078091F1049091F20490931A0780938F
:1073800019078091EF049091F00490931C0780936B
:107390001B0780911C04A090DC07B090DD07C09013
:1073A000DE07D090DF078823A9F08091B70790917E
:1073B000B807AA2797FDA095BA2FBC01CD010E945E
:1073C000EE42DC01CB01A6019501BC01CD010E947A
:1073D00068433AC080917A0490917B04A0917C0428
:1073E000B0917D04BC01CD010E94EE427B018C0175
:1073F0008091CC079091CD07A091CE07B091CF0797
:107400009C01AD01C801B7010E9468437B018C015A
:107410008091B7079091B807AA2797FDA095BA2F3A
:10742000BC01CD010E94EE42DC01CB01A601950119
:10743000BC01CD010E946843DC01CB019C01AD0180
:10744000C801B7010E944942DC01CB01BC01CD015A
:107450000E94D142DC01CB019093B8078093B7071B
:1074600080911B04A090DC07B090DD07C090DE0780
:10747000D090DF078823A9F08091AD079091AE07E7
:10748000AA2797FDA095BA2FBC01CD010E94EE421C
:10749000DC01CB01A6019501BC01CD010E9468432E
:1074A0003AC08091720490917304A0917404B091D9
:1074B0007504BC01CD010E94EE427B018C018091DC
:1074C000CC079091CD07A091CE07B091CF079C013A
:1074D000AD01C801B7010E9468437B018C01809116
:1074E000AD079091AE07AA2797FDA095BA2FBC01D2
:1074F000CD010E94EE42DC01CB01A6019501BC0149
:10750000CD010E946843DC01CB019C01AD01C801A3
:10751000B7010E944942DC01CB01BC01CD010E94B0
:10752000D142DC01CB019093AE078093AD078091EF
:10753000D8079091D907AA2797FDA095BA2FBC012B
:10754000CD010E94EE427B018C018091DC0790917D
:10755000DD07A091DE07B091DF079C01AD01BC0102
:10756000CD010E944942DC01CB019C01AD01C80163
:10757000B7010E9468437B018C0180915E04909169
:107580005F04A0916004B0916104BC01CD010E9430
:10759000EE42DC01CB014090CC075090CD076090CB
:1075A000CE077090CF07A3019201BC01CD010E94CC
:1075B0006843DC01CB0120E030E040E05FE3BC0148
:1075C000CD010E946843DC01CB019C01AD01C801E3
:1075D000B7010E944942DC01CB01BC01CD010E94F0
:1075E000D142DC01CB019093D9078093D8078091D9
:1075F000B7079091B8079093080780930707809189
:10760000AD079091AE0790930A0780930907809188
:10761000B7079091B8078150904434F080E090E42F
:107620009093B8078093B7078091B7079091B807F8
:107630008050904C34F480E090EC9093B8078093A5
:10764000B7078091AD079091AE078150904434F018
:1076500080E090E49093AE078093AD078091AD07F2
:107660009091AE078050904C34F480E090EC909371
:10767000AE078093AD078091D8079091D9078150CC
:10768000904434F080E090E49093D9078093D80739
:107690008091D8079091D9078050904C34F480E0C5
:1076A00090EC9093D9078093D80789819A81880FAD
:1076B000991F880F991F9A83898380916D07992755
:1076C00080FFF0C020917E0381FF0EC0223310F5B1
:1076D00080912304909124044497909322048093F2
:1076E000210410923A0419C080917203909173039F
:1076F000820F911D209172073327829FD001839FB3
:10770000B00D929FB00D1124CD01449790932204A7
:107710008093210481E080933A04BB81BB2321F054
:107720001092220410922104009123041091240449
:107730002091210430912204201731070CF0B2C0AF
:1077400080913A04882309F4ADC0021B130B809189
:107750007D039927089FF001099FF00D189FF00DF8
:107760001124CF01F7FD03968C011595079515950A
:107770000795E980FA80E01AF10A87018091D90320
:107780009091DA0397FD019695958795081B190B43
:10779000C0904204D0904304E0904404F09045042B
:1077A000F7FE08C02FE730E040E050E0C20ED31EE5
:1077B000E41EF51EA7E0F594E794D794C794AA9524
:1077C000D1F780917C03282F332744275527C70101
:1077D000B6010E94B04397FF04C0615E7F4F8F4F98
:1077E0009F4FF5E09595879577956795FA95D1F731
:1077F00031E0693173071CF068E171E006C04EEFBB
:10780000683E740714F468EE7EEF061B170B809138
:10781000BD049091BE049C01E4E0220F331FEA9561
:10782000E1F7281B390B200F311F37FF02C0215F02
:107830003F4F74E0359527957A95E1F73093BE0474
:107840002093BD0480916E07482F5527440F551F84
:10785000440F551F2417350794F489819A818417A2
:10786000950724F05093BE044093BD04A981BA81CA
:10787000A417B50724F4B093BE04A093BD0480916F
:10788000BD049091BE04E981FA81E817F90724F458
:10789000F093BE04E093BD04E090BD04F090BE04FC
:1078A000FA82E9823090D707832D9927880F991F94
:1078B000880F991F8055904009811A818017910780
:1078C00014F49A83898329813A813093EC062093BA
:1078D000EB068091A4049091A504A091A604B09118
:1078E000A70442E0880F991FAA1FBB1F4A95D1F732
:1078F0008090D8079090D907881A990A213A3105C3
:107900008CF0C90137FD01969595879588159905E5
:107910000CF44C01909581959F4F8816990694F42C
:107920004C0110C031E5831691041CF010E5812E46
:10793000912C40EB84164FEF940624F4B0EB8B2E81
:10794000BFEF9B2E232D3327220F331F220F331F10
:10795000C901A981BA818A1B9B0B881599050CF472
:107960004C01E981FA81E21BF30B8E169F060CF4A1
:107970004F018091B7079091B807E0902C04F090E8
:107980002D04FD8AEC8A8E199F099093C10780937C
:10799000C00720E030E040E050E0C301B2010E94A7
:1079A000F84220919C0430919D0440919E04509196
:1079B0009F04882309F448C0CA01B9010E94EE421D
:1079C0005B016C0180917A0490917B04A0917C040E
:1079D000B0917D04BC01CD010E94EE42DC01CB01DF
:1079E000A3019201BC01CD010E9468437B018C017F
:1079F0002C893D89C901AA2797FDA095BA2FBC0102
:107A0000CD010E94EE42DC01CB019C01AD01C80119
:107A1000B7010E944842DC01CB019C01AD01C601C7
:107A2000B5010E944942DC01CB01BC01CD010E949D
:107A3000D142DC01CB0180939C0490939D04A093E0
:107A40009E04B0939F0414C08091C0079091C10719
:107A5000AA2797FDA095BA2F280F391F4A1F5B1F31
:107A600020939C0430939D0440939E0450939F0464
:107A700080919C0490919D04A0919E04B0919F04DC
:107A800081509A4FA040B04064F080E09AEFA0E0AF
:107A9000B0E080939C0490939D04A0939E04B093C7
:107AA0009F0480919C0490919D04A0919E04B091AC
:107AB0009F0480509640AF4FBF4F64F480E096E043
:107AC000AFEFBFEF80939C0490939D04A0939E041E
:107AD000B0939F048091C0079091C107AA2797FD9A
:107AE000A095BA2FBC01CD010E94EE427B018C0112
:107AF00080919C0490919D04A0919E04B0919F045C
:107B0000BC01CD010E94EE42DC01CB01209180033B
:107B1000309181034091820350918303288B398BEC
:107B20004A8B5B8B9C01AD01688979898A899B8925
:107B30000E946843DC01CB019C01AD01C801B70183
:107B40000E944942DC01CB01BC01CD010E94D1421F
:107B5000DC01CB018C0120907403622D77278827EC
:107B60009927940197FE04C0222733272819390941
:107B700037FF02C02F5F3F4F3595279549815A81C6
:107B8000240F351F442737FD4095542F0E94B043E2
:107B900097FF04C0615C7F4F8F4F9F4FE6E0959544
:107BA000879577956795EA95D1F79B0160177107DF
:107BB0000CF48B01309521953F4F021713070CF4FD
:107BC000890129813A81200F311F280D391DC901F2
:107BD00037FD03969C01359527953595279537FFF9
:107BE00003C020E030E006C0832D99278217930759
:107BF0000CF49C013090B907832D99272817390779
:107C00000CF49C012093AF0729813A81201B310B92
:107C1000280D391DC90137FD03969C01359527951F
:107C20003595279537FF03C020E030E007C08091ED
:107C3000D7079927821793070CF49C01832D992766
:107C4000281739070CF49C012093B6078091AD07E3
:107C50009091AE07A0912A04B0912B04BD8BAC8B00
:107C60008A1B9B0B9093AC078093AB0720E030E01E
:107C700040E050E0C301B2010E94F8422091A0040C
:107C80003091A1044091A2045091A304882309F4E7
:107C900048C0CA01B9010E94EE425B016C018091AB
:107CA000720490917304A0917404B0917504BC01A6
:107CB000CD010E94EE42DC01CB01A3019201BC0187
:107CC000CD010E9468437B018C01EC89FD89CF01C5
:107CD000AA2797FDA095BA2FBC01CD010E94EE42C4
:107CE000DC01CB019C01AD01C801B7010E944842F3
:107CF000DC01CB019C01AD01C601B5010E944942E6
:107D0000DC01CB01BC01CD010E94D142DC01CB01E1
:107D10008093A0049093A104A093A204B093A30421
:107D200014C08091AB079091AC07AA2797FDA0954E
:107D3000BA2F280F391F4A1F5B1F2093A0043093CE
:107D4000A1044093A2045093A3048091A0049091B5
:107D5000A104A091A204B091A30481589E43A04025
:107D6000B04064F080E89EE3A0E0B0E08093A0041F
:107D70009093A104A093A204B093A3048091A004C3
:107D80009091A104A091A204B091A3048058914CB9
:107D9000AF4FBF4F64F480E891ECAFEFBFEF80933B
:107DA000A0049093A104A093A204B093A304809193
:107DB000AB079091AC07AA2797FDA095BA2FBC01FD
:107DC000CD010E94EE427B018C018091A004909134
:107DD000A104A091A204B091A304BC01CD010E9412
:107DE000EE42DC01CB019C01AD01688979898A8969
:107DF0009B890E946843DC01CB019C01AD01C80155
:107E0000B7010E944942DC01CB01BC01CD010E94B7
:107E1000D142DC01CB018C01622D7727882799277D
:107E2000940197FE04C0222733272819390937FF08
:107E300002C02F5F3F4F3595279549815A81240F06
:107E4000351F442737FD4095542F0E94B04397FFBC
:107E500004C0615C7F4F8F4F9F4F26E095958795BB
:107E6000779567952A95D1F79B01601771070CF4F8
:107E70008B01309521953F4F021713070CF48901B0
:107E800029813A81200F311F28193909C90137FD8D
:107E900003969C01359527953595279537FF03C0A7
:107EA00020E030E007C08091D70799278217930719
:107EB0000CF49C01832D9927281739070CF49C0199
:107EC0002093D20729813A81201B310B28193909C7
:107ED000C90137FD03969C01359527953595279562
:107EE00037FF03C020E030E007C08091D707992713
:107EF000821793070CF49C01832D992728173907C3
:107F00000CF49C012093D00765960FB6F894DEBF61
:107F10000FBECDBFDF91CF911F910F91FF90EF90DA
:107F2000DF90CF90BF90AF909F908F907F906F9099
:107F30005F904F903F902F9008958091E70490912B
:107F4000E804A091E904B091EA048093DF049093DF
:107F5000E004A093E104B093E2048091E3049091E3
:107F6000E404A091E504B091E6048093DB049093CF
:107F7000DC04A093DD04B093DE0408951092F204B3
:107F80001092F1041092F0041092EF04089584B15D
:107F9000806A84B93D9A82E58CBD1DBC459A81E01A
:107FA0008093E7078AEA8093EB0783E88093EC07E6
:107FB0008AE08093ED071092EF071092EE0710927F
:107FC000F1071092F00710920D080895F89480912F
:107FD0007A0490917B04A0917C04B0917D04BC0153
:107FE000CD012CE630E040E050E00E942444309384
:107FF000EF072093EE078091720490917304A09193
:108000007404B0917504BC01CD012CE630E040E071
:1080100050E00E9424443093F1072093F0078091B0
:10802000E1079091E207A091E307B091E407BC015A
:10803000CD012EE036E040E050E00E942444309331
:10804000F7072093F607E0918404F091850480916E
:10805000C6079091C707BF010E94EF432CE030E0B4
:10806000629FA001639F500D729F500D1124509389
:10807000F3074093F2078091DA079091DB07BF0185
:108080000E94EF43629FA001639F500D729F500DAD
:1080900011245093F5074093F40710928504109231
:1080A00084041092C7071092C6071092DB07109243
:1080B000DA078091ED0799278A30910561F08A30BF
:1080C00091050CF4A7C08B30910511F1821793072D
:1080D00009F497C09FC0809116048093FE07809199
:1080E00015048093FF078091140480930008809109
:1080F00013048093010880911204809302088091F8
:10810000110480930308809110048093040882C0B6
:1081100080916707E82FFF27EE0FFF1FE75CF84FFE
:108120000190F081E02DE038F1051CF0EFE7F0E080
:1081300006C05FEFE138F50714F4E1E8FFEFE093E4
:10814000FE0780916807E82FFF27EE0FFF1FE75C0F
:10815000F84F0190F081E02DE038F1051CF0EFE7D9
:10816000F0E006C06FEFE138F60714F4E1E8FFEF46
:10817000E093FF0780916607E82FFF27EE0FFF1FB0
:10818000E75CF84F0190F081E02DE038F1051CF03C
:10819000EFE7F0E006C08FEFE138F80714F4E1E80C
:1081A000FFEFE093000880916507E82FFF27EE0FAF
:1081B000FF1FE75CF84F0190F081E02DE038F105FA
:1081C0001CF0EFE7F0E006C02FEFE138F20714F4FF
:1081D000E1E8FFEFE0930108809135048093020805
:1081E00080913304809303088091310480930408C4
:1081F00080912F048093050880912E0480930608B7
:1082000009C080913606863018F01092360685E057
:108210008093FE07789480910D08882309F456C056
:1082200040910F0850911008CA0181509E4F8F5FF6
:108230009340B0F42091110830911208C901815087
:108240009E4F8F5F934060F480916D0785FF08C05B
:108250005093F2044093F1043093F0042093EF0420
:10826000809115089091160821E08936920724F430
:108270009093410480934004809140049091410484
:1082800020913E0430913F04821B930B845E9D4FEE
:1082900068E671E00E94EF43845B904090933D0458
:1082A00080933C0480911908282F33278091CD03B7
:1082B0009091CE038217930788F480913606882325
:1082C00069F43093CE032093CD0308951092F20405
:1082D0001092F1041092F0041092EF04089580912E
:1082E000E707882309F43BC045988BEE97E090930D
:1082F000E9078093E8079091F304E92FFF27E755FA
:10830000FC4F9F5F9093F30480818093ED0795303D
:1083100010F01092F3041092E7070E94E63F81E00C
:108320008093EA0700000000000000000000000049
:10833000000000000000000000000000000000003D
:10834000000000000000000000000000000000002D
:10835000000000008091EB0780930A088EBD08950D
:108360003091E707332309F085C00DB407FE82C0C2
:1083700084E08093CC03459A2EB58091F50499272B
:108380008130910589F0823091051CF4892B21F010
:108390003EC00297B9F03BC030930C082093F6041E
:1083A0002138A9F581E008C0253549F48091F6040B
:1083B000820F8093F60482E08093F50428C0309306
:1083C000F50425C080910C08E82FFF27E95DF74FE1
:1083D00020838F5F80930C089091F6048931A0F080
:1083E000291769F4AEE0B8E0E7E2F8E089E101902E
:1083F0000D928150E1F781E080930D0802C0309327
:108400000D081092F50403C0920F9093F60420918A
:10841000EA07203208F028C045980000000000005C
:10842000000000000000000000000000000000004C
:10843000000000000000000000000000000000003C
:1084400000000000000000000000E091E807F0914B
:10845000E907E20FF11D80818EBD80910A089081AD
:10846000890F80930A0803C081E08093E7072F5F9C
:108470002093EA070895FC014150504030F00190EC
:108480000616D1F73197CF010895882799270895C7
:108490005058192EEFD001D0D2C0BA176207730717
:1084A00084079507B1F188F40EF410940B2EBA2FBF
:1084B000A02D062E622F202D072E732F302D082E73
:1084C000842F402D092E952F502DFF275523B9F0CD
:1084D000591B49F0573E98F0469537952795A79533
:1084E000F0405395C9F776F0BA0F621F731F841FCF
:1084F00030F4879577956795B795F040939517FA7F
:108500000F2E0895BF1BBB27BA0B620B730B840B96
:10851000F6CFDEF6DBC0AED001D091C0552359F0C6
:10852000992369F09F575F57951B33F442F49038B5
:1085300011F4915805C09BC091589F3F09F4C6C0E3
:10854000BB27112462177307840730F4660F771F67
:10855000881FBB1F915098F311D00F920FD00F922C
:108560000DD0A0E82617370748071B0609F0A048DA
:10857000BA2F602D7F918F9100240895A0E80024E8
:10858000621773078407B10528F0621B730B840B15
:10859000B1090A2A660F771F881FBB1FA69581F7AE
:1085A000089597FB73D09F3738F0FEE9F91B982F99
:1085B000872F762F6B2F05C086C096958795779568
:1085C0006795F150D0F73EF4909580957095619540
:1085D0007F4F8F4F9F4F0895E89403C097FB0EF491
:1085E000F3DFB62F672F782F892F9EE9002427C04D
:1085F0000ED05EF004C00BD026F001C008D019F0F8
:1086000020F48FEF089580E0089581E0089597FBAE
:10861000092E052600F8689430D0E89407FC07C0BE
:10862000621773078407950721F008F400940794F4
:10863000989408959A95BB0F661F771F881F112481
:108640009923A1F08823B2F79F3F59F0BB0F48F45C
:1086500021F4002011F460FF04C06F5F7F4F8F4F43
:108660009F4F881F9795879597F908952CC09FEF86
:1086700080EC0895052E092607FA440F551F5F3F29
:1086800079F0AA27A51708F051E04795880F991FA0
:108690009F3F31F0BB27B91708F091E08795089507
:1086A0009F919F911124E3CF97FB880F991F9F3FC4
:1086B00031F0BB27B91708F091E0879508959F9195
:1086C0009F911124D4CF662777278827992708956B
:1086D000D1DF01D0B4CF992339F0552329F09F572A
:1086E0005F57950F13F49AF1F1CF91589F3FE1F343
:1086F000629FA12D0F92BB27639FA00DB11DEE2796
:10870000729FA00DB11DEE1FAF93AA27649FB00DFD
:10871000E11D739FB00DE11DAA1F6627829FB00D5A
:10872000E11DA61F5527749FE00DA11D551F839FB6
:10873000E00DA11D561F849FA00D511D852F7A2F7E
:108740006E2F1F900F9088231AF4939539F48FCFD2
:10875000000C111CBB1F661F771F881F012808957E
:10876000629FD001739FF001829FE00DF11D649F15
:10877000E00DF11D929FF00D839FF00D749FF00DA1
:10878000659FF00D9927729FB00DE11DF91F639F42
:10879000B00DE11DF91FBD01CF0111240895991BF2
:1087A00079E004C0991F961708F0961B881F7A95E8
:1087B000C9F780950895AA1BBB1B51E107C0AA1FEA
:1087C000BB1FA617B70710F0A61BB70B881F991F72
:1087D0005A95A9F780959095BC01CD01089597FB16
:1087E000092E07260AD077FD04D0E5DF06D0002049
:1087F0001AF4709561957F4F0895F6F790958195DD
:108800009F4F0895A1E21A2EAA1BBB1BFD010DC0AC
:10881000AA1FBB1FEE1FFF1FA217B307E407F50730
:1088200020F0A21BB30BE40BF50B661F771F881F0C
:10883000991F1A9469F760957095809590959B01A2
:10884000AC01BD01CF01089597FB092E05260ED07E
:1088500057FD04D0D7DF0AD0001C38F4509540955E
:10886000309521953F4F4F4F5F4F0895F6F7909504
:108870008095709561957F4F8F4F9F4F0895F9991F
:10888000FECFB2BDA1BDF89A119600B40895F99932
:10889000FECFB2BDA1BD00BC11960FB6F894FA9AF6
:0688A000F99A0FBE0895D5
:1088A600010A01496E74656772616C4E69636B20DB
:1088B600202020496E74656772616C526F6C6C2063
:1088C6002020204163634E69636B202020202020F6
:1088D600202020416363526F6C6C202020202020D2
:1088E6002020204779726F4769657220202020205A
:1088F600202020486F6568656E57657274202020B9
:108906002020204163635A20202020202020202080
:108916002020204761732020202020202020202096
:108926002020204B6F6D7061737356616C756520E6
:108936002020205370616E6E756E672020202020E7
:10894600202020456D7066616E6720202020202043
:1089560020202045727361747A6B6F6D706173733A
:108966002020204D6F746F725F566F726E652020E7
:108976002020204D6F746F725F48696E74656E209B
:108986002020204D6F746F725F4C696E6B732020D0
:108996002020204D6F746F725F5265636874732078
:1089A6002020204163635F5A2020202020202020A1
:1089B60020202044697374616E6365202020202086
:1089C6002020204F73644261722020202020202026
:1089D6002020204D4B334D61672043616C537461F9
:1089E600746520536572766F202020202020202079
:1089F6002020204E69636B2020202020202020206C
:108A0600202020526F6C6C20202020202020202047
:108A16002020202020202020202020202020202050
:108A26002020202020202020202020202020202040
:108A36002020202020202020202020202020202030
:108A46002020202020202020202020202020202020
:108A56002020202020202020202020202020202010
:108A66002020202020202020202020202020202000
:108A760020202020202020202020202020202020F0
:108A86002020204750535F4E69636B202020202012
:108A96002020204750535F526F6C6C2020202020EE
:108AA60020202064FF01FFFF280001806400FF03EF
:108AB600007D0000640048616C6C6F2057656C7423
:108AC60000000000000000000000000000000000A0
:108AD6000000000000000000000000000000000090
:108AE6000000000000000000000000000000000080
:108AF6000000000000000000000000000000000070
:108B06000000000000000102030405060708090A28
:108B16000B01ECFF6446640A029696403A10FB305D
:108B260017B7D13890D0030090D00300F401640049
:108B360053706F727400004E6F726D616C0000426C
:0E8B46006567696E6E657200000A0B0A0B0C03
:00000001FF
